:020000020000FC
:100000000C94874D1895189518951895189518956E
:100010001895189518951895189518951895189578
:100020001895189518951895189518951895189568
:100030001895189518951895189518950C94F92FEA
:1000400018951895189518950C94024918951895B7
:100050001895189518951895189518951895189538
:100060001895189518951895189518951895189528
:1000700018951895189518950C94DC4818951895AE
:100080001895189518951895189518950D0A20002B
:100090000D0A0A205B434D2D352056657273696F3A
:1000A0006E20312E31345D000D0A20546F737320A1
:1000B0004D6F64650D0A000D0A202D3E5B44796E7C
:1000C000616D6978656C5D3A000D0A203C2D5B44DA
:1000D000796E616D6978656C5D3A000D0A203C2D82
:1000E0003E50433A00203C2D3E44796E616D697864
:1000F000656C3A000D0A2041726520796F75207396
:10010000757265203F28792F4E29000D0A205573FE
:10011000616765203A20476F205B506F736974698F
:100120006F6E20416E676C6528307830307E307895
:10013000336666295D000D0A20416C6C2044796E9F
:10014000616D6978656C27732049442077696C6C10
:100150002062652073657420746F20002E20417228
:100160006520796F7520737572653F28592F4E2968
:10017000000D0A204572726F72315B436865636BD4
:100180002044796E616D6978656C2056657273697B
:100190006F6E206973206D6F7265207468616E20C8
:1001A000335D000D0A2042284265666F7265292C76
:1001B0004E284E657874292C512851756974290090
:1001C0000D0A203438354D6F6E69746F72205B4CA8
:1001D000462C43522061726520616464656420612D
:1001E000742070617573652074696D655D0D0A001A
:1001F0000D0A204E6F20446174615B61742042726D
:100200006F61646361737420494420307846455DB2
:10021000000D0A204E6F20446174612843686563B5
:100220006B2049442C204F7065726174696E6720A1
:100230004D6F64652C20426175642072617465297C
:1002400000204C454E3A000D0A204C454420426C9B
:10025000696E6B2049443A002044796E616D69787B
:10026000656C7320466F756E642E000D0A204C4538
:100270004420426C696E6B2049443A000D20466F61
:10028000756E642120424155445F5245473A002C27
:100290002049443A000D0A20426175642052656786
:1002A000206973206368616E67656420746F200045
:1002B000425053000D0A2049443A30202D20000DB1
:1002C0000A2044656C61793A000D0A20546F7271FE
:1002D000756520456E61626C65000D0A204D6F7674
:1002E000652030203C2D3E203078336666000D0AB4
:1002F00020416E79204B657920746F20436F6E74B6
:10030000696E75652E2E2E000D0A205B45455052F4
:100310004F4D20415245415D0D0A204D4F44454C03
:100320005F4E554D4245525F4C202020202020201A
:1003300020285229205B000D0A204D4F44454C5F78
:100340004E554D4245525F4820202020202020203D
:10035000285229205B000D0A2056455253494F4E22
:100360002020202020202020202020202020202885
:100370005229205B000D0A20494420202020202003
:100380002020202020202020202020202028522F24
:1003900057295B000D0A20424155445F52415445A4
:1003A00020202020202020202020202028522F57CD
:1003B000295B000D0A2052455455524E5F44454C6E
:1003C00041595F54494D452020202028522F57295C
:1003D0005B000D0A2043575F414E474C455F4C4937
:1003E0004D49545F4C202020202028522F57295B54
:1003F000000D0A2043575F414E474C455F4C494D25
:1004000049545F48202020202028522F57295B0084
:100410000D0A204343575F414E474C455F4C494DC1
:1004200049545F4C2020202028522F57295B000D73
:100430000A204343575F414E474C455F4C494D4965
:10044000545F482020202028522F57295B000D0A96
:10045000202852455345525645442920202020202B
:1004600020202020202028522F57295B000D0A2011
:100470004C494D49545F54454D5045524154555295
:10048000452020202028522F57295B000D0A2044A8
:100490004F574E5F4C494D49545F564F4C5441475E
:1004A0004520202028522F57295B000D0A20555047
:1004B0005F4C494D49545F564F4C544147452020AD
:1004C00020202028522F57295B000D0A204D41582B
:1004D0005F544F525155455F4C2020202020202052
:1004E000202028522F57295B000D0A204D41585FCC
:1004F000544F525155455F48202020202020202075
:100500002028522F57295B000D0A2052455455527E
:100510004E5F4C4556454C20202020202020202096
:1005200028522F57295B000D0A20414C41524D5F44
:100530004C4544202020202020202020202020283E
:10054000522F57295B000D0A20414C41524D5F53F9
:10055000485554444F574E20202020202020285218
:100560002F57295B000D0A20285245534552564506
:100570004429202020202020202020202028522F05
:1005800057295B000D0A20444F574E5F43414C49A9
:1005900042524154494F4E5F4C20202028522F5741
:1005A000295B000D0A20444F574E5F43414C49429E
:1005B000524154494F4E5F4820202028522F57293E
:1005C0005B000D0A2055505F43414C494252415453
:1005D000494F4E5F4C202020202028522F57295B66
:1005E000000D0A2055505F43414C49425241544945
:1005F0004F4E5F48202020202028522F57295B0093
:100600000D0A205B52414D20415245415D0D0A20AB
:10061000544F525155455F454E41424C4520202094
:10062000202020202028522F57295B000D0A204C23
:100630004544202020202020202020202020202071
:100640002020202028522F57295B000D0A204357D5
:100650005F434F4D504C49414E43455F4D415247DA
:10066000494E2028522F57295B000D0A204343573B
:100670005F434F4D504C49414E43455F4D415247BA
:10068000494E28522F57295B000D0A2043575F43DC
:100690004F4D504C49414E43455F534C4F504520C0
:1006A0002028522F57295B000D0A204343575F43F0
:1006B0004F4D504C49414E43455F534C4F504520A0
:1006C00028522F57295B000D0A20474F414C5F509D
:1006D0004F534954494F4E5F4C2020202020202862
:1006E000522F57295B000D0A20474F414C5F504F56
:1006F000534954494F4E5F48202020202020285243
:100700002F57295B000D0A204D4F56494E475F5326
:10071000504545445F4C2020202020202028522F87
:1007200057295B000D0A204D4F56494E475F5350E5
:100730004545445F482020202020202028522F5764
:10074000295B000D0A20544F525155455F4C494DCD
:1007500049545F4C2020202020202028522F572948
:100760005B000D0A20544F525155455F4C494D498D
:10077000545F482020202020202028522F57295B1A
:10078000000D0A2050524553454E545F504F534977
:1007900054494F4E5F4C20202020285229205B00D6
:1007A0000D0A2050524553454E545F504F53495403
:1007B000494F4E5F4820202020285229205B000D01
:1007C0000A2050524553454E545F53504545445FAF
:1007D0004C20202020202020285229205B000D0AB8
:1007E0002050524553454E545F53504545445F4851
:1007F00020202020202020285229205B000D0A20C4
:1008000050524553454E545F4C4F41445F4C20205D
:10081000202020202020285229205B000D0A205073
:10082000524553454E545F4C4F41445F4820202071
:100830002020202020285229205B000D0A20505221
:100840004553454E545F564F4C5441474520202058
:1008500020202020285229205B000D0A20505245DC
:1008600053454E545F54454D5045524154555245A1
:10087000202020285229205B000D0A20524547499C
:100880005354455245445F494E53545255432E20CC
:100890002028522F57295B000D0A205245534552FC
:1008A0005645442850415553455F54494D452920EC
:1008B00028522F57295B000D0A204D4F56494E47AD
:1008C0002020202020202020202020202020202028
:1008D000285229205B000D0A204C4F434B2020203A
:1008E00020202020202020202020202020202852CE
:1008F0002F57295B000D0A2050554E43485F4C206E
:100900002020202020202020202020202028522F9E
:1009100057295B000D0A2050554E43485F48202060
:1009200020202020202020202020202028522F5747
:10093000295B000D0A0A2044554D50284429203ACD
:100940002044756D7020636F6E74726F6C207461DB
:10095000626C652E000D0A204944205B49445F4EBD
:10096000554D5D203A20536574204944206F662020
:1009700064796E616D6978656C2E000D0A204349BB
:1009800044205B49445F4E554D5D203A20436861E9
:100990006E676520436F6E74726F6C2049442E0041
:1009A0000D0A2052454144205B414444525D5B4C5A
:1009B000454E5D203A205265616420646174612E69
:1009C0002065782952656164203130203220285218
:1009D0006561642066726F6D20307831302C206C38
:1009E000656E677468203229000D0A2057524954F9
:1009F00045205B414444525D5B44415441315D2E8E
:100A00002E203A20577269746520646174612E202B
:100A100065782957726974652031342C3120285744
:100A20007269746520312061742030783134290076
:100A30000D0A205245475F5752205B414444525DA6
:100A40005B44415441315D2E2E203A205265676946
:100A50007374657220777269746520696E7374753A
:100A6000726374696F6E000D0A20414354494F4E02
:100A7000203A20416374696F6E205245475F575298
:100A800020696E737472756374696F6E000D0A204D
:100A9000476F205B504F534954494F4E5D5B535055
:100AA0004545445D3A20476F746F20746865207037
:100AB0006F736974696F6E207769746820746865F4
:100AC0002073706565642E000D0A20484558205B30
:100AD0004E554D5D5B4E554D5D2E2E2E203A2054C9
:100AE00072616E736D6974652072617720646174E0
:100AF000612E2065782948657820464620464620A4
:100B00003031203033000D0A205245534554203AED
:100B10002044796E616D6978656C205265736574E7
:100B20002E000D0A2050494E47205B4E554D5D3A30
:100B3000206578292050696E67204E554D20494424
:100B40002064796E616D6978656C2E000D0A205302
:100B50005752205B414444525D5B4C454E5D5B49BE
:100B6000445D5B444154415D2E2E2E5B49445D5BE8
:100B7000444154415D2E2E2E203A2053796E63203D
:100B800057726974652E000D0A205343414E205B55
:100B90004E554D5D203A205343414E206C696E6B9B
:100BA00065642064796E616D6978656C20696E207A
:100BB000307E4E554D20696E2063757272656E747D
:100BC000206261756420726174652E000D0A204CEC
:100BD0004544205B4E554D5D203A20426C696E6B5A
:100BE000204C4544206F66204E554D2049442E2010
:100BF0002742272C274E2720666F72204944206306
:100C000068616E67652E2027512720666F7220511C
:100C10007569742E000D0A2042415544205B4E55E3
:100C20004D5D203A205365742062617564207261C5
:100C300074652020657829204241554420323228AD
:100C40003537363030425053292C2042415544200C
:100C50003128314D42505329000D0A20534541524D
:100C60004348203A205365617263682049442061FB
:100C70006E64206261756472617465206F662061C4
:100C80006C6C206C696E6B65642064796E616D6953
:100C900078656C732E000D0A2055706461746520B0
:100CA0005B53544152545F49445D205B454E445F61
:100CB00049445D203A2044796E616D6978656C2005
:100CC0006669726D77617265207570646174652EF6
:100CD0002873797374656D2075736572206F6E6CFF
:100CE0007929000D0A0A2020202020202020436F8F
:100CF0007079726967687420524F424F544953208B
:100D0000434F2E2C4C54442E0D0A005B496E7661E5
:100D10006C6964205061676520526561643A000D1A
:100D20000A205B4572723A5278442054696D656FAF
:100D300075745D000D0A205B4572723A57726F6ED2
:100D400067204865616465725D000D0A205B45722D
:100D5000723A5478494420213D20527849445D003C
:100D60000D0A205B4572723A57726F6E67204C65B0
:100D70006E6774685D000D0A205B4572723A5772A7
:100D80006F6E6720436865636B53756D5D000D0A78
:100D900020555044415445205B53544152542049FE
:100DA000445D205B454E442049445D005D3A000DA2
:100DB0000A2049443A00205374616E6462792E001F
:100DC0002057726974696E672E2E00205375636315
:100DD0006573732E00204572726F722E000D0A200B
:100DE0004572722049443A002042616420436F6D8D
:100DF0006D616E64005B457869745D005B53544FB0
:100E0000505D000D0A204D4F54494F4E20504C412B
:100E10005920504147452020202028522F57290093
:100E20000D0A204F4E20504C4159494E47204D4FFE
:100E300054494F4E2020202028522920000D0A20FE
:100E4000545820574952454C455353205041434B29
:100E50004554202028522F5729000D0A205258208F
:100E6000574952454C455353205041434B4554201C
:100E7000202028522920000D0A204E45572050419D
:100E8000434B455420415252495645442020202886
:100E9000522920000D0A20415558204C454420205D
:100EA000202020202020202020202028522F5729B9
:100EB000000D0A20425554544F4E282D532D552DC8
:100EC000442D4C2D522920202028522920000D0A83
:100ED0002054494D4552283132356D5365632045C4
:100EE000616368292028522F5729000D0A205A498A
:100EF0004742454520494420202020202020202012
:100F0000202028522F5729000D0A20524F424F54BB
:100F1000204944202020202020202020202020287C
:100F2000522F5729000D44796E616D6978656C20E8
:100F300020302830783030295B202020205D000DC3
:100F40000A44796E616D6978656C202031283078AB
:100F50003031295B202020205D0020506167654EE4
:100F6000756D6265723A000D0A44796E616D69783B
:100F7000656C2020322830783032295B20202020F8
:100F80005D0020416464723A000D0A44796E616D1F
:100F90006978656C2020332830783033295B202035
:100FA00020205D00202852657365727665642920D3
:100FB0003A000D0A44796E616D6978656C202034C1
:100FC0002830783034295B202020205D002020202C
:100FD000506C6179436F756E743A000D0A44796EF6
:100FE000616D6978656C2020352830783035295B53
:100FF000202020205D00202852657365727665648C
:1010000029203A000D0A44796E616D6978656C207B
:1010100020362830783036295B202020205D0020C3
:1010200028526573657276656429203A000D0A447A
:10103000796E616D6978656C20203728307830379B
:10104000295B202020205D00202852657365727680
:10105000656429203A000D0A44796E616D697865EE
:101060006C2020382830783038295B202020205D03
:10107000002028526573657276656429203A000D58
:101080000A44796E616D6978656C20203928307862
:101090003039295B202020205D002020205061670E
:1010A0006520537465703A000D0A44796E616D696C
:1010B00078656C2031302830783041295B20202041
:1010C000205D0020436F6E74726F6C436F64653AED
:1010D000000D0A44796E616D6978656C20313128A4
:1010E00030783042295B202020205D002020506194
:1010F00067652053706565643A000D0A44796E6136
:101100006D6978656C2031322830783043295B2056
:101110002020205D0020202044584C205365747509
:10112000703A000D0A44796E616D6978656C203102
:10113000332830783044295B202020205D00202097
:10114000416363656C2054696D653A000D0A44790A
:101150006E616D6978656C203134283078304529AE
:101160005B202020205D004C696E6B20746F204E48
:101170006578743A000D0A44796E616D6978656C22
:101180002031352830783046295B202020205D0032
:101190004C696E6B20746F20457869743A000D0AB3
:1011A00044796E616D6978656C203136283078310C
:1011B00030295B202020205D0028526573657276FF
:1011C00065645031293A000D0A44796E616D697881
:1011D000656C2031372830783131295B2020202080
:1011E0005D002852657365727665645231293A0054
:1011F0000D0A44796E616D6978656C20313828304C
:10120000783132295B202020205D002852657365EB
:10121000727665645032293A000D0A44796E616D28
:101220006978656C2031392830783133295B20208A
:1012300020205D00285265736572766564523229FC
:101240003A000D0A44796E616D6978656C20323020
:101250002830783134295B202020205D000D0A449D
:10126000796E616D6978656C20323128307831355E
:10127000295B202020205D000D0A44796E616D6994
:1012800078656C2032322830783136295B20202076
:10129000205D000D0A44796E616D6978656C2032BD
:1012A000332830783137295B202020205D000D0A5B
:1012B00044796E616D6978656C20323428307831FC
:1012C00038295B202020205D000D0A44796E616D75
:1012D0006978656C2032352830783139295B2020D7
:1012E00020205D000D0A44796E616D6978656C207F
:1012F00032362830783161295B202020205D000DB6
:101300000A44796E616D6978656C203237283078CF
:101310003162295B202020205D000D0A44796E6136
:101320006D6978656C2032382830783163295B200C
:101330002020205D000D0A44796E616D6978656C2E
:101340002032392830783164295B202020205D004C
:101350000D0A44796E616D6978656C2033302830F0
:10136000783165295B202020205D000D0A20202097
:10137000506175736554696D652020202020202000
:101380005B2020205D000D0A2020205370656564DD
:101390002020202020202020202020000D0A202096
:1013A0002054696D6528207820372E386D53656389
:1013B00029005B2020205D202020202020202020CC
:1013C000202020202020202020202020202020201D
:1013D00020202020202020202020205B583A2D2D66
:1013E0002C593A2D2D2C413A2D2D2D2D5D000D0A15
:1013F00020202020202020202020202020202020ED
:101400002020205354503720205354503020535420
:1014100050312053545032205354503320535450A1
:101420003420535450352053545036202020204728
:101430006F20537465703A2020202020000D0A2070
:10144000202020202020202020202020202020209C
:1014500020202020202020204D53545220534C4146
:1014600056204F465354202020202020202020208A
:101470002020202020202020202020202020476FF6
:1014800020537465703A2020202020000D0A5D2032
:101490005F2020202020202020202020202020200D
:1014A000202020202020202020202020202020203C
:1014B000202020202020202020202020202020202C
:1014C000202020202020202020202020202020201C
:1014D0002020202020202020202000204172652074
:1014E000796F7520737572653F5B792F4E5D0020B3
:1014F000496E76616C696420506167650020496EB1
:1015000076616C696420506172616D65746572000A
:10151000204F66667365742055706461746564005D
:10152000204F7574206F662052616E676500204FF2
:101530004B000D0A20202020202020202D434D3A52
:101540002052503D2850617261302C4F502C506118
:1015500072613129204C4B205253205B414444524C
:101560005D2020000D0A20427265616B20617420AD
:10157000000D0A204552524F523A00494620202081
:10158000202000454C534520494600454C534520FA
:10159000202000616E642F6F7220004A554D50204C
:1015A0002020004C4F414420202000434F4D5055F7
:1015B0005445005354415254202000454E442020AD
:1015C00020200043414C4C202020005245545552CD
:1015D0004E20004E554C4C202020000D0A2048453E
:1015E000584120444953504C4159204D4F444500E7
:1015F0000D0A20444543494D414C20444953504C29
:101600004159204D4F44450003404C464D4840450C
:101610004A230102030A222121217D7D7D7D7D7DDA
:101620007D7D7D7D7D7D7D7D7D797673716E6C693F
:1016300067656361605E5C5B595857555453515000
:101640004F4E4D4C4B4A4948474645444342424120
:10165000403F3F3E3D3C3C3B3A39393837373636E0
:10166000353434333332313130302F2F2E2D2D2C71
:101670002C2B2B2A2A2929282827272626252525E9
:1016800024242323222221212020201F1F1E1E1D4F
:101690001D1D1C1C1B1B1A1A1A19191818181717AC
:1016A0001616161515141414131312121211111004
:1016B00010100F0F0E0E0E0D0D0C0C0C0B0B0A0A5A
:1016C00009090908080707070606050504040403B5
:1016D0000302020101010000000000000000000000
:1016E00000000000000000000000000000000000FA
:1016F00000000000000000000000000000000000EA
:1017000000000000000000000000000000000000D9
:1017100000000000000000000000000000010101C6
:1017200002000200010101010200010101010200A9
:101730000200010101010101020002000200020099
:101740000200020001010101010102000101020089
:10175000020000000001010101010000010101017E
:101760000100010101010101000001010000000070
:101770000000010000000101020001010000010160
:101780000101020002000101682FA901812F00233D
:10179000B9F40FE003BF00E002BF09E01DE30E94BF
:1017A000DF4D10E0003021E0120710F000E009C02A
:1017B00001BF082F00FB07B701F907BF01E001C017
:1017C00000E0862F089500E00093610002B901BB9C
:1017D00004BB07BB0ABB00E00093650000936200F6
:1017E00003B902BB05BB08BB00B50B7F00BD00B54C
:1017F0000B7F00BD00E00093610002B901BB04BB98
:1018000007BB0ABB00E0009365000093620003B9C8
:1018100002BB05BB08BBBD9AC59A909A1C9A1D9A3B
:101820001E9A1F9A04B30F6704BB02B10C6002B981
:10183000AC9AAB9AAA9AA99AA89AAE9AAD9AAC9A7F
:10184000AB9AAA9AA99AA89A1A981B9A01B3006708
:1018500001BB9798949A959A9698AC9AAB9AAA9A43
:10186000A99AA89A0895002391F400E000939000AB
:1018700019B902E00BB908E10AB920FB0EF4579A36
:1018800006E0009395000FEF0CB95E9A08950130C1
:10189000E9F400E0009398001093990002E00093AF
:1018A0009B0008E100939A0020FB2EF400919A001F
:1018B000006800939A0006E000939D000FEF0093EC
:1018C0009C0000919B00006400939B000895592F99
:1018D000482F80E090E008C02FE93FE021503040E1
:1018E000E9F700C00000019680179107A8F3842F44
:1018F000952F08959A938A9380E090E098D20A33C6
:1019000018F00753102F02C00053102F012F10E0C2
:10191000102F00E0110F110F110F110F802B912BC1
:1019200086D20A3318F00753102F02C00053102F2D
:10193000012F302F20E0822B932B79D20A3318F01D
:101940000753102F02C00053102F012F10E044E066
:101950000E94D34D802B912B6AD20A3318F0075383
:10196000102F02C00053102F012F10E0802B912B5D
:101970008C018991999108950E94754E24972A832C
:101980003B83B02FD12E7A0182E090E001E00093FA
:10199000F30CBB249699B394CC249599C394969A4E
:1019A000959825C0949801E010E091DF00E0009345
:1019B000090D0093080D949A05E010E088DF01E21C
:1019C00005D101E311E083DF08E000D10091080DAB
:1019D0001091090D011751F00091080D1091090D9A
:1019E000011721F024D20132B9F791E08A958130B4
:1019F00010F09923B9F2992309F4B1C000E00093E3
:101A0000090D0093080D4424552466247724A0E092
:101A10008824992409E6DAD008E0D8D008D20A331D
:101A2000E9F705D2088303D2098301D20A33E9F723
:101A300061DF2801FCD10A33E9F75CDF3801088156
:101A4000003319F40981063431F002E6BFD000E317
:101A5000BDD006E6BBD00FEF60160FEF700649F061
:101A6000E6D10A33E9F7E3D1093511F4A1E001C069
:101A7000A0E00EE110E02BDF00E00093090D0093E1
:101A8000080D02E5A3D008E0A1D0D1D1802F8C367B
:101A900041F4CDD10A33E9F72DDF4801AA24A394FC
:101AA00003C08F3691F7AA24EDEEFCE0408251820C
:101AB000EFEEFCE060827182E1EFFCE080829182D7
:101AC000B0FBC6F404E110E002DF04E47FD008E0DC
:101AD0007DD0ADD10A33E9F705E010E0F8DE0A81E8
:101AE0001B817BD108E072D008E070D008E06ED096
:101AF00008E06CD0B1FB4EF404E110E0E8DEDA1649
:101B000021F007E563D008E061D0B2FBCEF4AA2053
:101B1000B9F004E110E0DBDE03E458D008E056D071
:101B200086D10A33E9F705E010E0D1DE870155D10F
:101B300008E04CD008E04AD008E048D008E046D0A1
:101B400004E110E0C4DE05E441D008E03FD0949801
:101B500001E010E0BCDE949A04E610E0B8DE00E09C
:101B60000093090D0093080D0B2D00FD969A00FFC0
:101B700096980C2D00FD959A00FF959800E0009333
:101B8000F30C092F2496E0E10C94864E5E9A1B9884
:101B90001A9A18D05E9BFECF1A981B9A08958A93C2
:101BA000802F082F02950F70005D0A3308F0095F3F
:101BB0000DD08F70805D082F0A3308F0095F06D0C2
:101BC000899108955D9BFECF0CB90895A998109155
:101BD0009B00212F25FFFBCF00939C0008959A9333
:101BE0008A93802F082F44E60E94B54D902F092F2D
:101BF000005DECDF04E6909F8019082F4AE00E9408
:101C0000B54D902F092F005DE1DF0AE0909F80190C
:101C1000805D082FDBDF8991999108950E94774EAE
:101C200048015901DD24BB2052F49094A094B09453
:101C3000000B8194900AA00AB00A0DE2C7DF80E091
:101C40009AECAAE9BBE3CC241AC0DD2019F082018A
:101C5000005DBCDF82019301AC01BD010E94044E16
:101C6000801A910AA20AB30A8C019D014AE050E051
:101C700060E070E00E944E4EC801D901C39409E0B3
:101C8000C016A8F484019501AC01BD010E944E4E1E
:101C9000402E552466247724042D0529062907297A
:101CA000A1F28201005D92DFDD24D394D3CF8401C1
:101CB0009501AC01BD010E944E4E402E5524662474
:101CC0007724042D005D82DFEEE00C94884E0E94A4
:101CD0007D4E38015524A0E1B7E244240FC000E353
:101CE00075DF8C01AD010E94C34D601A710A8D0130
:101CF0004AE050E00E94DF4DD801439405E04016D1
:101D0000D0F48301AD010E94DF4DC801082F092BDB
:101D100031F0082F005D5ADF55245394E2CF55204F
:101D200021F0082F005D52DFDCCF04E04016B8F64A
:101D300000E24CDFD6CFE8E00C948E4E10916A0999
:101D4000112311F02CDF089523E010E00AD008954C
:101D500020916A09222311F040D0089524E001D097
:101D600008950E947B4E3801822E5524A0E1B7E2EF
:101D700044240FC000E32ADF8C01AD010E94C34D53
:101D8000601A710A8D014AE050E00E94DF4DD801CF
:101D9000439405E04016F0F48301AD010E94DF4D4D
:101DA000C80104E010E0242D30E0021B130B99243D
:101DB000081519050CF7082F092B31F0082F005DC5
:101DC00005DF55245394D8CF5520A1F2082F005D8C
:101DD000FDDED2CFEAE00C948C4E9A938A93C80130
:101DE0008C01012F10E0DBDE082FD9DE899199915B
:101DF00008950E94814EC801D9018C019D01022FD6
:101E0000132F330F220B330BE8DF8C01E6DFE4E006
:101E10000C94924EBA93AA93D80103C00C91D6DECB
:101E200011960C910023D1F7A991B99108950091D1
:101E3000090D1091080D0117D1F30091090D102F14
:101E400013951093090D10E00F701070F801E65F04
:101E5000F24F008108958A93802F082FC0DE08E298
:101E6000B5DE00E3B3DE08E5B1DE082F98DE09E257
:101E7000ADDE899108950E947A4EEF97EF97EF9724
:101E80002797A898992401E00093730901E0009333
:101E9000720905C004E110E01ADD08E001BD9920D7
:101EA00011F00C94131803EA15E0B4DF00916309F4
:101EB000D2DF0CEA15E0AEDF20E08E0108571F4F9D
:101EC0000E94C41F00E00883AE0148575F4F9E0187
:101ED000205F3F4F8E010E94181E802E00917009D6
:101EE000009371098820D9F20FE1801610F00EE1FD
:101EF000802E28E536E08E010E94F61D002351F663
:101F000026E536E08E010E94F61D002309F450C03C
:101F100007EB10E00E940D4C80E01CC0FE017096A3
:101F2000082F10E0000F111F000F111FE00FF11F0D
:101F3000008111812281338190E0FC01EA52F74F48
:101F4000008390E0FC01EA52F74F0081F7DE00E2E7
:101F50003DDE839590E0E82DF0E031978E179F07E6
:101F6000ECF21B981A9A80E008C090E0FC01EA525B
:101F7000F74F008127DE5E9A839590E0E82DF0E030
:101F800031978E179F078CF35E9BFECF1A981B9A92
:101F90000FEF0E94B2490093740909EC10E00E940F
:101FA0000D4C2091740902E218E00E94BF4A77CFDD
:101FB00021E536E08E010E94F61D002371F42EE427
:101FC00036E08E010E94F61D002339F421EA35E047
:101FD0008E010E94F61D002369F100916309083CFF
:101FE000B1F40CE810E00E940D4C088919892A8987
:101FF0003B8931DF0AE3EADD088919892A893B89AF
:10200000102F009163090E94A53CA2DE48CF0889E9
:1020100019892A893B890093A0070C891D892E897B
:102020003F890093A10722E012E0009163090E941A
:10203000E94A35CF2CE935E08E010E94F61D0023D8
:10204000A9F014E3009163090E945C4DC801282F98
:1020500014E1009163090E94901D892F90E0282FC0
:1020600015E1009163090E94901D19CF27E935E021
:102070008E010E94F61D002331F114E300916309E3
:102080000E945C4DD80114E1009163090E945C4DEF
:10209000C80116E1009163090E945C4D080F191FE9
:1020A000169507950A1B1B0B212F27FF04C00195CE
:1020B000006810E001C010E0202F1AE000916309D1
:1020C0000E94901DECCE23E935E08E010E94F61DA2
:1020D000002341F001E000936A090BED15E10E9435
:1020E0000D4CDDCE2FE835E08E010E94F61D002359
:1020F00041F000E000936A0900EF15E10E940D4CE9
:10210000CECE2AE835E08E010E94F61D0023A9F00C
:1021100014E3009163090E945C4DC801282F16E169
:10212000009163090E94901D892F90E0282F17E1EC
:10213000009163090E94901DB2CE26E835E08E0121
:102140000E94F61D002339F42EE735E08E010E942F
:10215000F61D0023F9F080E014C0FE017096082FF0
:1021600010E0000F111F000F111FE00FF11F008181
:1021700011812281338190E0FC01E056F84F008309
:102180008395881550F38A94282D13E80EEF0E944A
:10219000E94A85CE28E735E08E010E94F61D00232E
:1021A00071F425E735E08E010E94F61D002339F415
:1021B00023E735E08E010E94F61D0023A1F1009176
:1021C0006309083C81F40C891D892E893F89980197
:1021D000488959896A897B898A01102F009163098E
:1021E0000E94923B5CCE80E014C0FE017096082FE6
:1021F00010E0000F111F000F111FE00FF11F0081F1
:1022000011812281338190E0FC01E056F84F008378
:102210008395881550F38A94282D13E00091630963
:102220000E94E94A3CCE2CE635E08E010E94F61D64
:10223000002301F180E014C0FE017096082F10E029
:10224000000F111F000F111FE00FF11F00811181FE
:102250002281338190E0FC01E056F84F00838395A2
:10226000881550F38A94282D14E0009163090E9488
:10227000E94A15CE25E635E08E010E94F61D0023C1
:1022800039F421E635E08E010E94F61D0023F9F0B5
:1022900080E014C0FE017096082F10E0000F111F9F
:1022A000000F111FE00FF11F008111812281338186
:1022B00090E0FC01E056F84F00838395881550F3B9
:1022C0008A94282D15E00EEF0E94E94AE8CD2AE510
:1022D00035E08E010E94F61D002381F00C891D89D6
:1022E0002E893F89202F488959896A897B898A01EB
:1022F000102F009163090E94901DD1CD24E535E097
:102300008E010E94F61D002321F104EF10E00E94CF
:102310000D4C8DDD093719F0093509F0C0CD01E00C
:10232000801619F40091630904C0088919892A8963
:102330003B8920E016E00E94E94A002309F4AFCD72
:1023400001E00093630921E030E0A9010E94B14D52
:10235000A6CD2DE435E08E010E94F61D0023A1F0EC
:1023600001E0801639F420E017E0009163090E9433
:10237000E94A95CD20E017E0488959896A897B8927
:10238000042F0E94E94A8BCD2AE435E08E010E9499
:10239000F61D002339F428E435E08E010E94F61D75
:1023A0000023D9F102E0801619F003E0801681F5D0
:1023B0000EE10093A007088919892A893B890093B7
:1023C000A107088919892A893B89012F10E0009308
:1023D000A20703E08016A9F40C891D892E893F8984
:1023E0000093A3070C891D892E893F89012F10E0D6
:1023F0000093A40725E013E0009163090E94E94AD5
:102400004ECD23E013E0009163090E94E94A47CDD5
:102410000BE011E00E940D4C42CD23E435E08E012B
:102420000E94F61D002379F001E0801619F4009156
:10243000630904C0088919892A893B8920E011E0D1
:102440000E94E94A2CCD20E435E08E010E94F61D61
:10245000002349F103E00093A007088919892A891C
:102460003B890093A10706E311E00E940D4C009107
:10247000A10764DC0CE511E00E940D4CD8DC0935A5
:1024800019F0093709F00BCD22E013E00EEF0E949E
:10249000E94A0091A1070093630921E030E0A90116
:1024A0000E94B14DFCCC2AE036E08E010E94F61D60
:1024B000002339F428E036E08E010E94F61D002347
:1024C000E1F000916309083C11F400D6E8CC00E08B
:1024D0000093A0070AE30093A10722E012E0009115
:1024E00063090E94E94A002309F4D9CC00916309E9
:1024F0000E3F09F4D4CCEAD5D2CC21E036E08E01EF
:102500000E94F61D002309F4A5C103E0801651F4D2
:10251000488859886A887B880C891D892E893F895B
:10252000A02E0DC002E0801631F4488859886A88D0
:102530007B88A42C04C00EE81DE00E940D4C02E034
:10254000801621F003E0801609F0A9CC00E000938A
:1025500072090093730909B1023289F421E014E091
:102560000EEF0E94724D0AE010E0B1D901E009B906
:102570000093620920E030E0A9010E94B14D22E2FF
:1025800014E00EEF0E94724D0AE010E0A0D902E2C2
:1025900009B90093620920E030E0A9010E94B14D21
:1025A00021E014E00EEF0E94724D0AE010E08FD996
:1025B00001E009B90093620920E030E0A9010E941E
:1025C000B14D00E00E94284C05C001E711E00E94D7
:1025D0000D4C4394A41408F41EC15524F201EB5889
:1025E000F64F00810023A9F309B1013049F001E061
:1025F00009B90093620920E030E0A9010E94B14DC1
:102600000FEA1DE00E940D4C042D98DB90E0992309
:1026100099F491E080E08F31D0F7082F0E94C81D17
:10262000002341F020E011E0082F0E94E94A002336
:1026300009F490E08395EFCF06EB1DE00E940D4C6E
:1026400080E00FC0841561F090E0FC01EB58F64F7C
:102650000081002329F025E01DE2082F0E94901D33
:1026600083958F3178F300EC1DE00E940D4C2FEF25
:102670001AEF042D0E94901D2EEF1DE2042D0E94E2
:10268000901D002309F4A1CF03E0502E02E209B906
:102690000093620920E030E0A9010E94B14D04E6F8
:1026A00010E015D90DE072DA00E00E944A1D0CE43A
:1026B0006DDA00E00E944A1D1B981A9A80E090ECA7
:1026C000A0E0B0E088246624772412C0FC013A2FF1
:1026D0003BBF069000E00BBF8F5F9F4FAF4FBF4FD8
:1026E000800C002D6FDA5E9A01E0600E00E0701E33
:1026F0000FEF601607E1700648F3082D63DA5E9A63
:102700005E9BFECF1A981B9A00E00E944A1D06E5C8
:102710003DDA00E00E944A1D00E001C00395043646
:1027200038F410E0F801EE5DF74F10811D32B1F77B
:102730000395202F01C00395043638F410E0F8010A
:10274000EE5DF74F10811D32B1F7039510E001C027
:102750001395183090F4602F062F0395422F242FE5
:10276000239570E0FB01EE5DF74F308150E0FA01F8
:10277000EE5DF74F4081341759F3183031F50BEC0B
:102780001DE00E940D4C01E401DA00E00E944A1DA8
:1027900007E4FCD900E00E944A1D04E610E097D847
:1027A00001E009B90093620920E030E0A9010E942C
:1027B000B14D20E017E0042D0E94E94A0CE211E03F
:1027C00086D800E00093720904CF05ED1DE00E9459
:1027D0000D4C5A9409F063CF01E4D8D900E00E946F
:1027E0004A1D07E4D3D900E00E944A1D04E610E028
:1027F0006ED801E009B90093620920E030E0A90138
:102800000E94B14D20E017E0042D0E94E94A0CE23D
:1028100011E05DD8DECE21E014E00EEF0E94724D93
:102820000AE010E054D801E009B90093620920E001
:1028300030E0A9010E94B14D0E94D64B09B100932E
:10284000620920E030E0A9010E94B14D01E000934F
:10285000730925CB2CEF35E08E010E94F61D002375
:1028600009F440C0B091720900E00093730900932D
:10287000720980E001E0801611F4AEEF05C008890E
:1028800019892A893B89A02F0CE810E00E940D4C81
:1028900090E005C00DE29AD90DE598D993959A1765
:1028A00088F40BE593D9092F49DA0AE38FD920E0A0
:1028B00011E0092F0E94E94A002361F30FE486D951
:1028C0008395EACF0CE810E00E940D4C082FC3DA84
:1028D00008E512E00E940D4CB093720901E00093EC
:1028E0007309DDCA28EF35E08E010E94F61D002332
:1028F00009F450C001E0801619F4A091630905C0E5
:10290000088919892A893B89A02F01E0009372095F
:1029100000E00093730903EA11E00E940D4C80E08F
:1029200007E412E00E940D4C0A2F08DA0091090D0D
:102930001091080D011791F07ADA802F823411F08E
:10294000823609F4AA958E3411F08E3609F4A395D7
:102950000BE612E00E940D4C0A2FF0D921E019E19C
:102960000A2F0E94724D04E610E00E94670C20E0DE
:1029700019E10A2F0E94724D04E610E00E94670CD4
:10298000813521F0813711F08B3181F601E0009320
:10299000730985CA21EF35E08E010E94F61D0023E0
:1029A00009F48EC000E0009373090AE00FD980E0BB
:1029B00001C083958E3F08F078C089B920E011E00E
:1029C0000EEF0E94E94A0DE001D980FB1EF40BE2F4
:1029D000FDD802C00AE2FAD800917409002309F474
:1029E0005DC0A0E056C0B0E0FD01EE5DF74F008194
:1029F0000F3F09F04DC00A2F10E00F5F1F4FF80185
:102A0000EE5DF74F00810F3F09F042C00A2F10E042
:102A10000D5F1F4FF801EE5DF74F00810230C1F5E9
:102A20000A2F10E00E5F1F4FF801EE5DF74F408157
:102A300050E00A2F10E00D5F1F4FF801EE5DF74FD9
:102A4000208130E0240F351F0A2F10E00B5F1F4F4D
:102A5000F801EE5DF74F008110E0020F131F0F3FEA
:102A600020E01207A9F40CE712E00E940D4C082F99
:102A700065D90FE812E00E940D4C0A2F10E00E5F9E
:102A80001F4FF801EE5DF74F008158D90AE09ED83C
:102A9000A39500917409A01708F4A5CF0091090D22
:102AA0001091080D011709F484CF0091620909B94A
:102AB00001E0009373090DE089D800E287D8EFC9DF
:102AC0002CEE35E08E010E94F61D002391F104E00A
:102AD0000093A007088919892A893B890093A107D7
:102AE00022E013E00EEF0E94E94A05E912E00E949D
:102AF0000D4C00E814E82EE130E0488959896A89D4
:102B00007B894F5F5F4F6F4F7F4F0E94284E86D863
:102B100000EB12E00E940D4C088919892A893B8933
:102B200009B90093620920E030E0A9010E94B14D8B
:102B3000B6C924EE35E08E010E94F61D002309F48B
:102B400042C001E0801631F400E1402E5524662495
:102B5000772404C0488859886A887B8800EC11E093
:102B60000E940D4C2BC00091710910917009011742
:102B7000A1F080E090E0A0E0B0E0AA24009171090B
:102B800010E0F801E056F94F0081E1E7F9E010812B
:102B900013951083D3D800E219D88F5F9F4FAF4FA2
:102BA000BF4F84159505A605B705E8F2AA2031F4B4
:102BB0000DE00CD80AE00AD8AA24A39480E090E0A3
:102BC000A0E0B0E0EECF2FED35E08E010E94F61DC3
:102BD000002309F44AC0488859886A887B888C8910
:102BE0009D89AE89BF8904EB12E00E940D4C042D33
:102BF000A5D80FEB12E00E940D4C8C01A9D809EC6E
:102C000012E00E940D4CA0E006C021E018E10A2F5E
:102C10000E94724DA3954A16C0F70AED12E00E9479
:102C20000D4C0CC02FEF33E01EE10A2F0E947A4DAD
:102C3000A3954A16B8F78C010E94670C0091090D04
:102C40001091080D011709F02AC9A0E007C020E083
:102C500030E01EE10A2F0E947A4DA3954A16B8F77C
:102C60008C010E94670CA0E0E4CF2BED35E08E01D3
:102C7000BDD7002309F434C100E00093730900912B
:102C800063090093A00721E015E00EEF0E94E94AD6
:102C900001E0801641F520E130E0A9010E94A54D38
:102CA000802E80E090E0E82DF0E031978E179F07AE
:102CB0000CF042C0E82FF0E07196AF010E94A54DE4
:102CC00010E020E030E0FE017096482F50E0440F05
:102CD000551F440F551FE40FF51F008311832283F6
:102CE00033838395DFCF05E1801610F004E1802E59
:102CF00020E130E0082DA9010E94B14D80E015C00F
:102D0000FE017096082F10E0000F111F000F111F19
:102D1000E00FF11F0081118122813381E82FF0E063
:102D20007196AF010E94B14D839590E0E82DF0E0DF
:102D300031978E179F0724F30CE810E00E940D4C8A
:102D40000BE50E94E60D80E004C00DE50E94E60D53
:102D5000839590E0E82DF0E031978E179F07DCF423
:102D6000FE017096082F10E0000F111F000F111FB9
:102D7000E00FF11F00811181228133810E949E0E9C
:102D800090E0E82DF0E032978E179F07F4F60DE201
:102D90000E94E60DDDCF0091090D1091080D01177D
:102DA00009F099C00CE810E00E940D4C80E019C0B9
:102DB000FE017096082F10E0000F111F000F111F69
:102DC000E00FF11F0081118122813381102F0091CA
:102DD00063090E944D4D0E949E0E00E20E94E60D86
:102DE000839590E0E82DF0E031978E179F079CF6D1
:102DF000FE017096082F10E0000F111F000F111F29
:102E0000E00FF11F0081118122813381083CF9F02C
:102E100000916309043688F1009163090E3668F564
:102E200002E517E1FE017096282F30E0220F331FD4
:102E3000220F331FE20FF31F4081518162817381A2
:102E400050E0040F151FF80104910230B1F4FE01A7
:102E50007096082F10E0000F111F000F111FE00FD8
:102E6000F11F0081118122813381102F00916309AC
:102E70000E94A53C0E94A80EB0CF0AE117E1FE0116
:102E80007096282F30E0220F331F220F331FE20FDE
:102E9000F31F408151816281738150E0040F151F3F
:102EA000F8010491023009F083CFFE017096082FDB
:102EB00010E0000F111F000F111FE00FF11F008124
:102EC000118122813381102F009163090E945C4D92
:102ED0000E94A80E82CF01E0009373090C944F0F5B
:102EE00026ED35E08E0182D6002389F14888598885
:102EF0006A887B888C899D89AE89BF8900E00093B0
:102F00007309A0E04A1698F021E018E10A2F0E9408
:102F1000724DA395F7CF2FEF33E01EE10A2F0E94E9
:102F20007A4DA3954A16B8F78C010E94670CA0E071
:102F300007C020E030E01EE10A2F0E947A4DA395E1
:102F40004A16B8F78C010E94670CA0E0EBCF22ED87
:102F500035E08E014BD6002369F0088919892A894A
:102F60003B890093630921E030E0A9010E94B14D43
:102F70000C944F0F2DEC35E08E0138D6002331F440
:102F80002BEC35E08E0132D6002321F00E9423493C
:102F90000C944F0F25EC35E08E0128D6002331F438
:102FA00023EC35E08E0122D6002321F00E94564901
:102FB0000C944F0F2EEB35E08E0118D6002319F03C
:102FC0003CD00C944F0F2AEB35E08E010FD6002336
:102FD00081F002E0801640F0088919892A893B892E
:102FE0000E9460410C944F0F01E00E9460410C94DC
:102FF0004F0F23EB35E08E01F9D5002331F42FEA92
:1030000035E08E01F3D5002321F0992493940C949C
:103010004F0F0CE810E00E940D4C08EE1DE00E94DE
:103020000D4C0C944F0F00E000937309EF96EF9650
:10303000EF962796EBE00C948B4E03E319E00E9489
:103040000D4C05E519E00E940D4C0BE719E00E94BC
:103050000D4C00EA19E00E940D4C09EE19E00E94A7
:103060000D4C00E31AE00E940D4C07E61AE00E94A6
:103070000D4C0DE81AE00E940D4C08EC1AE00E947D
:103080000D4C06E01BE00E940D4C02E21BE00E948A
:103090000D4C0CE41BE00E940D4C07E81BE00E9465
:1030A0000D4C0CEC1BE00E940D4C05E11CE00E9455
:1030B0000D4C09E51CE00E940D4C06E91CE00E9445
:1030C0000D4C03EE1CE00E940D4C08950E94814EB1
:1030D00000916309083C09F0B9C088E103E01EE0F3
:1030E0000E940D4C082F0E942B0F0AE30E94E60D50
:1030F000182F009163090E94A53C0E94A80E839599
:1031000000E21EE00E940D4C082F0E942B0F0AE3E4
:103110000E94E60D182F009163090E94A53C0E94B1
:10312000A80E83950DE31EE00E940D4C082F0E940F
:103130002B0F0AE30E94E60D182F009163090E94ED
:10314000A53C0E94A80E839583950AE51EE00E9487
:103150000D4C082F0E942B0F0AE30E94E60D182F3A
:10316000009163090E94A53C0E94A80E8395839557
:1031700007E71EE00E940D4C082F0E942B0F0AE368
:103180000E94E60D182F009163090E94A53C0E9441
:10319000A80E839504E91EE00E940D4C082F0E94A2
:1031A0002B0F0AE30E94E60D182F009163090E947D
:1031B000A53C0E94A80E839501EB1EE00E940D4CD9
:1031C000082F0E942B0F0AE30E94E60D182F009192
:1031D00063090E94A53C0E94A80E83950EEC1EE098
:1031E0000E940D4C082F0E942B0F0AE30E94E60D4F
:1031F000182F009163090E94A53C0E94A80E839598
:103200000BEE1EE00E940D4C082F0E942B0F0AE3CC
:103210000E94E60D182F009163090E94A53C0E94B0
:10322000A80E8395839508E01FE00E940D4C082F9F
:103230000E942B0F0AE30E94E60D182F00916309EC
:103240000E94A53C0E94A80E839521C480E008E05E
:1032500013E00E940D4C082F0E942B0F0CEA1DE07A
:103260000E940D4CA82FB0E01596FD01EE5DF74FC2
:1032700000810E942B0F839507E313E00E940D4C01
:10328000082F0E942B0F0CEA1DE00E940D4CA82F66
:10329000B0E01596FD01EE5DF74F00810E942B0F07
:1032A000839506E513E00E940D4C082F0E942B0F1A
:1032B0000CEA1DE00E940D4CA82FB0E01596FD0110
:1032C000EE5DF74F00810E942B0F839505E713E019
:1032D0000E940D4C082F0E942B0F0CEA1DE00E944B
:1032E0000D4CA82FB0E01596FD01EE5DF74F008163
:1032F0000E942B0F839504E913E00E940D4C082FC8
:103300000E942B0F0CEA1DE00E940D4CA82FB0E08C
:103310001596FD01EE5DF74F00810E942B0F8395FE
:1033200003EB13E00E940D4C082F0E942B0F0CEAB8
:103330001DE00E940D4CA82FB0E01596FD01EE5D3A
:10334000F74F00810E942B0F839502ED13E00E943E
:103350000D4C082F0E942B0F0CEA1DE00E940D4C13
:10336000A82FB0E01596FD01EE5DF74F00810E9499
:103370002B0F839501EF13E00E940D4C082F0E9444
:103380002B0F0CEA1DE00E940D4CA82FB0E0159603
:10339000FD01EE5DF74F00810E942B0F839500E148
:1033A00014E00E940D4C082F0E942B0F0CEA1DE028
:1033B0000E940D4CA82FB0E01596FD01EE5DF74F71
:1033C00000810E942B0F83950FE214E00E940D4CA8
:1033D000082F0E942B0F0CEA1DE00E940D4CA82F15
:1033E000B0E01596FD01EE5DF74F00810E942B0FB6
:1033F00083950EE414E00E940D4C082F0E942B0FC1
:103400000CEA1DE00E940D4CA82FB0E01596FD01BE
:10341000EE5DF74F00810E942B0F83950DE614E0BF
:103420000E940D4C082F0E942B0F0CEA1DE00E94F9
:103430000D4CA82FB0E01596FD01EE5DF74F008111
:103440000E942B0F83950CE814E00E940D4C082F6E
:103450000E942B0F0CEA1DE00E940D4CA82FB0E03B
:103460001596FD01EE5DF74F00810E942B0F8395AD
:103470000BEA14E00E940D4C082F0E942B0F0CEA5F
:103480001DE00E940D4CA82FB0E01596FD01EE5DE9
:10349000F74F00810E942B0F83950AEC14E00E94E5
:1034A0000D4C082F0E942B0F0CEA1DE00E940D4CC2
:1034B000A82FB0E01596FD01EE5DF74F00810E9448
:1034C0002B0F839509EE14E00E940D4C082F0E94EB
:1034D0002B0F0CEA1DE00E940D4CA82FB0E01596B2
:1034E000FD01EE5DF74F00810E942B0F839508E0F0
:1034F00015E00E940D4C082F0E942B0F0CEA1DE0D6
:103500000E940D4CA82FB0E01596FD01EE5DF74F1F
:1035100000810E942B0F839507E215E00E940D4C5D
:10352000082F0E942B0F0CEA1DE00E940D4CA82FC3
:10353000B0E01596FD01EE5DF74F00810E942B0F64
:10354000839506E415E00E940D4C082F0E942B0F76
:103550000CEA1DE00E940D4CA82FB0E01596FD016D
:10356000EE5DF74F00810E942B0F839505E615E075
:103570000E940D4C082F0E942B0F0CEA1DE00E94A8
:103580000D4CA82FB0E01596FD01EE5DF74F0081C0
:103590000E942B0F839504E815E00E940D4C082F24
:1035A0000E942B0F0CEA1DE00E940D4CA82FB0E0EA
:1035B0001596FD01EE5DF74F00810E942B0F83955C
:1035C00003EA15E00E940D4C082F0E942B0F0CEA15
:1035D0001DE00E940D4CA82FB0E01596FD01EE5D98
:1035E000F74F00810E942B0F839502EC15E00E949B
:1035F0000D4C082F0E942B0F0CEA1DE00E940D4C71
:10360000A82FB0E01596FD01EE5DF74F00810E94F6
:103610002B0F839501EE15E00E940D4C082F0E94A0
:103620002B0F0CEA1DE00E940D4CA82FB0E0159660
:10363000FD01EE5DF74F00810E942B0F83950EEE8A
:1036400012E00E940D4C0E94170F00E016E00E944D
:103650000D4C082F0E942B0F0CEA1DE00E940D4C10
:10366000A82FB0E01596FD01EE5DF74F00810E9496
:103670002B0F83950CE216E00E940D4C082F0E9440
:103680002B0F0CEA1DE00E940D4CA82FB0E0159600
:10369000FD01EE5DF74F00810E942B0F83950BE437
:1036A00016E00E940D4C082F0E942B0F0CEA1DE023
:1036B0000E940D4CA82FB0E01596FD01EE5DF74F6E
:1036C00000810E942B0F83950AE616E00E940D4CA4
:1036D000082F0E942B0F0CEA1DE00E940D4CA82F12
:1036E000B0E01596FD01EE5DF74F00810E942B0FB3
:1036F000839509E816E00E940D4C082F0E942B0FBD
:103700000CEA1DE00E940D4CA82FB0E01596FD01BB
:10371000EE5DF74F00810E942B0F839508EA16E0BB
:103720000E940D4C082F0E942B0F0CEA1DE00E94F6
:103730000D4CA82FB0E01596FD01EE5DF74F00810E
:103740000E942B0F839507EC16E00E940D4C082F6A
:103750000E942B0F0CEA1DE00E940D4CA82FB0E038
:103760001596FD01EE5DF74F00810E942B0F8395AA
:1037700006EE16E00E940D4C082F0E942B0F0CEA5B
:103780001DE00E940D4CA82FB0E01596FD01EE5DE6
:10379000F74F00810E942B0F839505E017E00E94F0
:1037A0000D4C082F0E942B0F0CEA1DE00E940D4CBF
:1037B000A82FB0E01596FD01EE5DF74F00810E9445
:1037C0002B0F839504E217E00E940D4C082F0E94F6
:1037D0002B0F0CEA1DE00E940D4CA82FB0E01596AF
:1037E000FD01EE5DF74F00810E942B0F839503E4EE
:1037F00017E00E940D4C082F0E942B0F0CEA1DE0D1
:103800000E940D4CA82FB0E01596FD01EE5DF74F1C
:1038100000810E942B0F839502E617E00E940D4C59
:10382000082F0E942B0F0CEA1DE00E940D4CA82FC0
:10383000B0E01596FD01EE5DF74F00810E942B0F61
:10384000839501E817E00E940D4C082F0E942B0F72
:103850000CEA1DE00E940D4CA82FB0E01596FD016A
:10386000EE5DF74F00810E942B0F839500EA17E071
:103870000E940D4C082F0E942B0F0CEA1DE00E94A5
:103880000D4CA82FB0E01596FD01EE5DF74F0081BD
:103890000E942B0F83950FEB17E00E940D4C082F11
:1038A0000E942B0F0CEA1DE00E940D4CA82FB0E0E7
:1038B0001596FD01EE5DF74F00810E942B0F839559
:1038C0000EED17E00E940D4C082F0E942B0F0CEA02
:1038D0001DE00E940D4CA82FB0E01596FD01EE5D95
:1038E000F74F00810E942B0F83950DEF17E00E9488
:1038F0000D4C082F0E942B0F0CEA1DE00E940D4C6E
:10390000A82FB0E01596FD01EE5DF74F00810E94F3
:103910002B0F83950CE118E00E940D4C082F0E949C
:103920002B0F0CEA1DE00E940D4CA82FB0E015965D
:10393000FD01EE5DF74F00810E942B0F83950BE395
:1039400018E00E940D4C082F0E942B0F0CEA1DE07E
:103950000E940D4CA82FB0E01596FD01EE5DF74FCB
:1039600000810E942B0F83950AE518E00E940D4C00
:10397000082F0E942B0F0CEA1DE00E940D4CA82F6F
:10398000B0E01596FD01EE5DF74F00810E942B0F10
:10399000839509E718E00E940D4C082F0E942B0F19
:1039A0000CEA1DE00E940D4CA82FB0E01596FD0119
:1039B000EE5DF74F00810E942B0F839508E918E018
:1039C0000E940D4C082F0E942B0F0CEA1DE00E9454
:1039D0000D4CA82FB0E01596FD01EE5DF74F00816C
:1039E0000E942B0F839507EB18E00E940D4C082FC7
:1039F0000E942B0F0CEA1DE00E940D4CA82FB0E096
:103A00001596FD01EE5DF74F00810E942B0F839507
:103A100006ED18E00E940D4C082F0E942B0F0CEAB7
:103A20001DE00E940D4CA82FB0E01596FD01EE5D43
:103A3000F74F00810E942B0F839505EF18E00E943D
:103A40000D4C082F0E942B0F0CEA1DE00E940D4C1C
:103A5000A82FB0E01596FD01EE5DF74F00810E94A2
:103A60002B0F839504E119E00E940D4C082F0E9452
:103A70002B0F0CEA1DE00E940D4CA82FB0E015960C
:103A8000FD01EE5DF74F00810E942B0F8395E4E06E
:103A90000C94924E9A938A93902F80E00091710932
:103AA000109170090117D1F340E050E060E070E040
:103AB00000917109109170090117A1F48A019B010D
:103AC000A801B9014F5F5F4F6F4F7F4F013EE3E9A0
:103AD0001E07E4E02E07E0E03E0750F3082F89912F
:103AE000999108950091710910E0F801E056F94F9D
:103AF0000081E1E7F9E0108113951083282F30E071
:103B0000F901EE5DF74F0083992341F0082F10E093
:103B1000F801EE5DF74F00810E94E60D8395C4CF5A
:103B20000E94814E902FA12FB22FA093A007B09397
:103B3000A10700EF0093A20705E50093A3070FE09C
:103B40000093A4070AEA0093A50726E01DE0092FC9
:103B50000E946E4A802F00917309002349F00CE8FF
:103B600010E00E940D4C282F06ED18E00E94BF4A7D
:103B700005E010E00E94670C1A2F092F0E944D4D9E
:103B80000B1711F401E001C000E0E4E00C94924E48
:103B90000F3130F410E0F801EB58F64F0081089532
:103BA000043650F00E3640F410E004561040F80190
:103BB000EB56F64F0081089500E00895A80100E05B
:103BC00001C00395083C88F410E0F901E00FF11FF3
:103BD000608110E0FA01E00FF11F608310E0F9014D
:103BE000E00FF11F1081112361F70895A80100E093
:103BF00010E0FA01E00FF11F608110E0F901E00F21
:103C0000F11F1081611791F4039510E0FA01E00FA4
:103C1000F11F1081112339F410E0F901E00FF11FB9
:103C20001081112321F0093C18F3089500E0089554
:103C30000E947E4ED901CA01442401C043945524F8
:103C4000FC01E40DF51D20812032C1F32CE3421666
:103C500008F041C05524FC01E40DF51D208122230C
:103C6000D1F120E021C05524FC01E40DF51D308187
:103C7000313670F05524FC01E40DF51D30813B37E1
:103C800038F45524FC01E40DF51D30813F75308377
:103C90005524FC01E40DF51D408130E0F801E20FF0
:103CA000F31F4083239543945524FC01E40DF51D37
:103CB0003081303350F05524FC01E40DF51D308186
:103CC0003B3718F430E1431670F240E030E0F80181
:103CD000E20FF31F4083E02FF12F0081002311F446
:103CE00000E0A6C066249EC043945524FC01E40D68
:103CF000F51D00810032C1F35524FC01E40DF51DD2
:103D00000081002319F46394062D92C000E010E0B6
:103D100020E030E0462D50E0440F551F440F551F62
:103D2000FD01E40FF51F008311832283338342C01A
:103D3000062D10E0000F111F000F111FFD01E00FF5
:103D4000F11F00811181228133814AE050E060E05F
:103D500070E00E94044E462D50E0440F551F440F62
:103D6000551FFD01E40FF51F008311832283338368
:103D70005524FC01E40DF51D008110E000531040B6
:103D8000212F220F220B322F462D50E0440F551FBA
:103D9000440F551FFD01E40FF51F408151816281E1
:103DA0007381400F511F621F731F408351836283D1
:103DB000738343940CE34016A0F55524FC01E40DF5
:103DC000F51D0081002321F402E0600E062D30C0B5
:103DD0005524FC01E40DF51D00810B33E1F0552461
:103DE000FC01E40DF51D00810A33A9F05524FC0106
:103DF000E40DF51D00810C3271F05524FC01E40D39
:103E0000F51D00810E3239F05524FC01E40DF51D3D
:103E10000081003281F400E25524FC01E40DF51D1F
:103E2000008363940EE1601608F45FCF6394062D5F
:103E3000E7E00C948F4E00916A09002309F478CFD3
:103E40005524FC01E40DF51D0081003308F446C043
:103E50005524FC01E40DF51D00810A33F8F5062D0B
:103E600010E0000F111F000F111FFD01E00FF11FE7
:103E7000008111812281338144E00E94204E462D31
:103E800050E0440F551F440F551FFD01E40FF51F6F
:103E900000831183228333835524FC01E40DF51D37
:103EA000008110E000531040212F220F220B322FEF
:103EB000462D50E0440F551F440F551FFD01E40FE0
:103EC000F51F4081518162817381400F511F621F34
:103ED000731F40835183628373836BCF5524FC012E
:103EE000E40DF51D0081013408F463CF5524FC0175
:103EF000E40DF51D00810B3708F05BCF5524FC0164
:103F0000E40DF51D00810F750083062D10E0000FF4
:103F1000111F000F111FFD01E00FF11F0081118122
:103F20002281338144E00E94204E462D50E0440F10
:103F3000551F440F551FFD01E40FF51F008311832A
:103F4000228333835524FC01E40DF51D008110E02C
:103F500007531040212F220F220B322F462D50E005
:103F6000440F551F440F551FFD01E40FF51F4081FD
:103F7000518162817381400F511F621F731F408303
:103F800051836283738315CF0E94814EC801A22F93
:103F9000B1E016C008E00E94E60D00E20E94E60DC6
:103FA00008E00E94E60D0A2FA02FAA95002391F7A2
:103FB00029EE3DE08C0102DEA02F8C010E940A0F49
:103FC000BB23A9F10E94170F102F1050C9F31A95A7
:103FD00051F3175099F0125029F0135019F01E5058
:103FE00079F319C000E0B0E0FC01EA0FFB1F008389
:103FF0009C0109EE1DE0E2DD01E01AC0A13000F3F2
:10400000AA9508E00E94E60D00E20E94E60D08E095
:104010000E94E60DD5CFAC3398F62A2F30E0FC0194
:10402000E20FF31F00830E94E60DA395C9CF00E0C5
:10403000E4E00C94924E0E94814E902F812F983094
:1040400050F5883040F5092F10E00F5F1F4F40E416
:1040500050E00E94C34DD801082F10E00F5F1F4FA2
:1040600040E450E00E94C34D20E011C0422F50E0D8
:10407000400F511FFA01E052F64F3081422F50E0BD
:104080004A0F5B1FFA01E052F64F3083239520342C
:1040900068F3092F03D0E4E00C94924E9A938A932C
:1040A000902F973011F490E001C0939580E007C005
:1040B000182F092F50D2182F092F2BD183958F310C
:1040C000B8F31FE1092F47D21FE1092FD3D0F80120
:1040D000E052F64F00810E949E0E10E2092F3BD263
:1040E00010E2092FC7D0F801E052F64F00810E947C
:1040F0009E0E899199910895005049F00A9561F0BA
:104100000A9579F00A9591F00A95A9F008950BEDBA
:1041100014E10E940D4C08950FEE14E10E940D4C25
:1041200008950DEF14E10E940D4C089500E115E192
:104130000E940D4C089500E215E10E940D4C089577
:104140009A938A93802F912FE7E1F6E11491EEE0A4
:10415000F6E104910E94C12F22E0082F10E00E9496
:10416000B10EE8E1F6E11491EFE0F6E104910E946E
:10417000C12F22E0092F10E00E94B10EE9E1F6E123
:104180001491E0E1F6E104910E94C12F192F082F4C
:1041900071D00E94A80E8991999108958A93E1E1C6
:1041A000F6E11491E8E0F6E104910E94C12F80E06D
:1041B00004C000E20E94E60D83958634D0F3E1E16D
:1041C000F6E11491E8E0F6E104910E94C12F899193
:1041D00008959A938A939091F40980E00CC0182F67
:1041E0000091250E0395B7D108E00E94E60D00E28C
:1041F0000E94E60D83958F3190F380E00BC0182F5D
:10420000092F0395A8D108E00E94E60D0CE70E9453
:10421000E60D83958F3198F39093250EE5E1F6E155
:104220001491ECE0F6E104910E94C12F092F0E9445
:104230009E0E899199910895093031F4133020F040
:10424000143110F401E00895083021F41F3110F406
:1042500001E00895083030F4103211F01F3111F4EC
:1042600001E00895083020F4103210F402E00895BF
:1042700000E00895682F202F812F222371F48F31C1
:1042800038F4082F10E0000F111F00501E4F39C0E6
:10429000082F10E0015E1D4F34C08F3149F4022F0A
:1042A00010E040E450E00E94C34D025C1F4F29C063
:1042B000803249F4022F10E040E450E00E94C34DE8
:1042C000015C1F4F1EC0283029F4082F10E0005E4B
:1042D0001F4F17C0293029F4082F10E0055F1F4F2A
:1042E00010C0022F10E00150104040E450E00E9446
:1042F000C34D980102E0809F8001020F131F005CF4
:104300001F4F003422E0120710F000E010E0862F6B
:1043100008959A938A93902F812F8F3108F042C08D
:10432000182F092FA7DFF801E052F64F20813181C5
:10433000203004E0300748F0182F092F9BDFF801E8
:10434000E052F64F018107FF0BC0182F092F92DFB3
:10435000F801E052F64F008111810E94A80E22C0A0
:10436000182F092F87DFF801E052F64F018105FF72
:104370000DC00FE30E94E60D0FE30E94E60D0FE370
:104380000E94E60D0FE30E94E60D0CC00DE20E94B4
:10439000E60D0DE20E94E60D0DE20E94E60D0DE233
:1043A0000E94E60D8991999108959A938A930091BC
:1043B000E50C002351F000E09FDE0E94170F093545
:1043C00021F0093711F000E085C0E3EEFCE0008148
:1043D000118120E030E040E052E060E070E00E94B7
:1043E000044EA801B901405050426F4F7F4F90E0FA
:1043F00000E010E018C0080122243324040E151E2A
:10440000261E371EF001322D3BBF069020E02BBF49
:10441000F801E052F64F0082F801E052F64F208199
:10442000920F0F5F1F4F003022E0120720F380E051
:104430000DC020E030E402E0809F800100501E4F5C
:10444000F801E052F64F2083318383958F3180F558
:10445000082F10E0F801EB58F64F0081002349F3D4
:1044600018E1082F0E944D4D013081F41EE1082F04
:104470000E94952F22E0829F20E0020E22E0121E71
:10448000F001E052F64F00831183DFCF14E2082FD2
:104490000E94952F0060106222E0829F20E0020EB1
:1044A00022E0121EF001E052F64F00831183CDCFBF
:1044B0009F3F21F40091F409083008F00ED000E08D
:1044C0000093E50C0091F709053018F000E0009327
:1044D000F70901E08991999108953B2F2A2FE0E097
:1044E000F0E006C000E0DF01A052B64F0C93319619
:1044F000E03200E0F007B0F3E0E2F0E006C005E5EE
:10450000DF01A052B64F0C933196E03400E0F00783
:10451000B0F3E0E4F0E009C000E010E4DF01A052F5
:10452000B64F0D931C9311973296E03002E0F007DE
:1045300098F300E00093F40901E00093EF0900E232
:104540000093F60900E20093F80900E00093ED09FA
:10455000A22FB32F08959A938A936297602F212FE9
:10456000CE010896EAEAFDE930E08C014AE050E02D
:104570000E94644ECE01E4EBFDE930E08C0148E09E
:1045800050E00E94644E203211F02F3151F42395F7
:10459000122FFE0170E0E60FF71F00810E94C12F6D
:1045A00010C02F3158F42395122FFE01389670E079
:1045B000E60FF71F00810E94C12F03C001E20E9495
:1045C000E60D62968991999108958A93802F03C090
:1045D00000E20E94E60D082F802F8A950023C1F784
:1045E000899108950E94824E80E005C00CE810E099
:1045F0000E940D4C83958C33C8F311E001E00E94BA
:10460000C12F05E21FE00E940D4C0FE31FE00E9446
:104610000D4C07E2DADF0AE51FE00E940D4C07E6C9
:104620001FE00E940D4C07E2D0DF02E81FE00E946D
:104630000D4C09E81FE00E940D4C07E2C6DF04EABA
:104640001FE00E940D4C02EB1FE00E940D4C07E2A0
:10465000BCDF0DEC1FE00E940D4C0BED1FE00E9433
:104660000D4C07E2B2DF06EF1FE00E940D4C04E0A4
:1046700010E10E940D4C07E2A8DF0FE110E10E945B
:104680000D4C0DE210E10E940D4C07E29EDF08E4A4
:1046900010E10E940D4C06E510E10E940D4C07E26E
:1046A00094DF01E710E10E940D4C0FE710E10E943A
:1046B0000D4C07E28ADF0AE910E10E940D4C08EA7E
:1046C00010E10E940D4C07E280DF03EC10E10E9434
:1046D0000D4C01ED10E10E940D4C07E276DF0CEE6F
:1046E00010E10E940D4C0AEF10E10E940D4C07E210
:1046F0006CDF05E111E10E940D4C03E211E10E9423
:104700000D4C07E262DF0EE311E10E940D4C0CE458
:1047100011E10E940D4C07E258DF07E611E10E940B
:104720000D4C05E711E10E940D4C07E24EDF00E958
:1047300011E10E940D4C0EE911E10E940D4C07E2BF
:1047400044DF09EB11E10E940D4C07EC11E10E94DE
:104750000D4C07E23ADF02EE11E10E940D4C00EF32
:1047600011E10E940D4C07E230DF0BE012E10E94E4
:104770000D4C09E112E10E940D4C07E226DF04E333
:1047800012E10E940D4C02E412E10E940D4C0DE575
:1047900012E10E940D4C08E712E10E940D4C03E962
:1047A00012E10E940D4C0EEA12E10E940D4C09EC40
:1047B00012E10E940D4C04EE12E10E940D4C0FEF2D
:1047C00012E10E940D4C0AE113E10E940D4C05E339
:1047D00013E10E940D4C00E513E10E940D4C0BE625
:1047E00013E10E940D4C0091F0090A3029F40CE904
:1047F00013E10E940D4C04C006E813E10E940D4C29
:1048000002EB13E10E940D4CE3EEFCE0008111810C
:10481000012B29F40DE314E10E940D4C04C00EEEAF
:1048200013E10E940D4C0CE814E10E940D4C80E055
:1048300001C083958132F8F490E006C0A23019F4EB
:10484000182F092F66DD9395933198F7182F092FAC
:10485000F3DCA02FAA23B9F3182F092F7CDEA13097
:1048600069F7182F092F06DDF801E052F64F008195
:104870000E949E0EE8CFADDCE2E1F6E11491E9E0A2
:10488000F6E104910E94C12F00EE19E00E940A0F88
:10489000E3E1F6E11491EAE0F6E104910E94C12F10
:1048A000E3EEFCE0008111810E94A80EE4E1F6E154
:1048B0001491EBE0F6E104910E94C12FE3EEFCE0DD
:1048C0000081118120E030E040E052E060E070E0E3
:1048D0000E94044E005010422F4F3F4F0E94F90E8D
:1048E000E3E00C94934E0E94784EEF97EA97DA95A6
:1048F000BE0164527F4FECEBFDE930E08B0141E2F9
:1049000050E00E94644EA0E0BA2FBA2ECA2E24EFC7
:104910003FE0A9010E94A54D053511F40C94DE2E4F
:104920001A2F0B2F0DDC1A2F0B2F15DE9090F40988
:1049300000916A09002319F000E1A02E02C00AE0EC
:10494000A02E0E94170F902F9B31D9F50E94170FB0
:10495000902F9B3519F40E94170F902F943421F457
:10496000BB2389F0BA950FC0933411F4B3950BC0F3
:10497000913421F4AA2339F0AA9505C0923419F490
:10498000A03208F4A395FE01E452FF4F0A2F10E075
:10499000E00FF11F00810B1738F4FE01E452FF4FC6
:1049A000B0E0EA0FFB1FB081BC1521F4AB1511F488
:1049B0000C94782F1A2F0B2FC3DBCB2EBA2E0C940E
:1049C000782F903209F044C01A2F0B2F35DC0230BB
:1049D00011F00C94782F80E090E21A2F0B2F4ADC14
:1049E000F801E052F64F0081118108271927008352
:1049F0001183BB2329F58A2F02E0809F800100509C
:104A00001E4FF801E052F64F018105FD16C090E0FF
:104A1000FC01EB58F64F0081002379F014E2082FD7
:104A20000E94952F22E0829F20E0020E22E0121EBB
:104A3000F001E052F64F008311830A2F0E94473A9B
:104A40001A2F0B2F66DC01E00093E50C0C94782FF5
:104A50009D3509F04CC01A2F0B2F7DDD1A2F0B2F1F
:104A6000EBDB0130B9F41A2F0B2F04DCF801E05214
:104A7000F64F0081039500831A2F0B2FFBDBF80103
:104A8000E052F64F00810E949E0E01E00093E50C7B
:104A90000C94782F023011F00C94782F1A2F0B2FD2
:104AA000E9DBF801E052F64F008111810F7F1370AE
:104AB0000F3F23E0120711F40C94782F1A2F0B2FBD
:104AC000D9DBF801E052F64F008111810F5F1F4FD3
:104AD000008311831A2F0B2F1CDCBB2319F40A2F20
:104AE0000E94473A01E00093E50C0C94782F9B3527
:104AF00009F04AC01A2F0B2F2EDD1A2F0B2F9CDB2B
:104B00000130B9F41A2F0B2FB5DBF801E052F64F44
:104B100000810A9500831A2F0B2FACDBF801E052BD
:104B2000F64F00810E949E0E01E00093E50C0C946C
:104B3000782F023011F00C94782F1A2F0B2F9ADB5C
:104B4000F801E052F64F008111810F7F1370012BA5
:104B500011F40C94782F1A2F0B2F8CDBF801E052F4
:104B6000F64F0081118101501040008311831A2FEC
:104B70000B2FCFDBBB2319F40A2F0E94473A01E029
:104B80000093E50C0C94782F9D3709F050C01A2F34
:104B90000B2F52DB0130B9F41A2F0B2F6BDBF8010E
:104BA000E052F64F00810A0D00831A2F0B2F62DBB3
:104BB000F801E052F64F00810E949E0E01E0009342
:104BC000E50C0C94782F023011F00C94782F1A2FEA
:104BD0000B2F50DBF801E052F64F008111810F7F5F
:104BE00013702FEF33E04A2D50E0241B350B0217D2
:104BF000130710F00C94782F8A2D90E01A2F0B2FAA
:104C000039DBF801E052F64F00811181080F191FBE
:104C1000008311831A2F0B2F7CDBBB2319F40A2F7F
:104C20000E94473A01E00093E50C0C94782F9B37E3
:104C300009F04CC01A2F0B2FFFDA0130B9F41A2FEC
:104C40000B2F18DBF801E052F64F00810A190083A0
:104C50001A2F0B2F0FDBF801E052F64F00810E9454
:104C60009E0E01E00093E50C0C94782F023011F0B9
:104C70000C94782F1A2F0B2FFDDAF801E052F64F23
:104C8000008111810F7F13702A2D30E00217130766
:104C900010F40C94782F8A2D90E01A2F0B2FEADA5B
:104CA000F801E052F64F00811181081B190B0083B7
:104CB00011831A2F0B2F2DDBBB2319F40A2F0E940F
:104CC000473A01E00093E50C0C94782F67DA9033B3
:104CD00060F09B3750F4092F0E94E60D98A721E061
:104CE0008E01085D1F4F50D905C020E08E01085D80
:104CF0001F4F4AD900E00883AE01485D5F4F9E0117
:104D00002C593F4F8E010E94181E902F992311F4A9
:104D10000C94782F23E935E08E010E94F61D0023C4
:104D200051F001E000936A09A0E0BA2F1A2F0B2F6F
:104D300007DA0C94782F29E436E08E010E94F61DE4
:104D4000002359F00AE00093F0094CDCA0E0BA2FF0
:104D50001A2F0B2FF5D90C94782F23E436E08E010F
:104D60000E94F61D002359F000E00093F0093ADCA0
:104D7000A0E0BA2F1A2F0B2FE3D90C94782F2FE82D
:104D800035E08E010E94F61D002351F000E00093F3
:104D90006A09A0E0BA2F1A2F0B2FD2D90C94782FC2
:104DA00020E436E08E010E94F61D002341F01ADC5B
:104DB000A0E0BA2F1A2F0B2FC3D90C94782F2CE315
:104DC00036E08E010E94F61D002339F424EE35E012
:104DD0008E010E94F61D002391F0E1E1F6E11491AD
:104DE000E8E0F6E104910E94C12F0E943B0FFADB3C
:104DF000A0E0BA2F1A2F0B2FA3D90C94782F27E3FA
:104E000036E08E010E94F61D0023B1F0933021F0B0
:104E100002E072D90C94782FFE01FF9605A116A12D
:104E200027A130A5B02FFE01FF9601A512A523A54D
:104E300034A5A02F0C94782F22E336E08E010E9437
:104E4000F61D002339F420E336E08E010E94F61DA2
:104E5000002349F1E3EEFCE0208131812F3700E0AF
:104E60003007E8F4E3EEFCE0008111810F5F1F4F93
:104E7000008311839ADA002341F0B4DBA0E0BA2F5B
:104E80001A2F0B2F5DD90C94782FE3EEFCE00081F4
:104E9000118101501040008311830C94782F01E0A0
:104EA0002BD90C94782F29E236E08E010E94F61D52
:104EB000002339F427E236E08E010E94F61D00231C
:104EC00021F1E3EEFCE000811181012BD9F0E3EE4A
:104ED000FCE000811181015010400083118365DAEC
:104EE000002339F07FDBA0E0BA2F1A2F0B2F28D92F
:104EF000FFC7E3EEFCE0008111810F5F1F4F0083CD
:104F00001183F6C701E0F8D8F3C722E236E08E013C
:104F10000E94F61D002339F420E236E08E010E9443
:104F2000F61D002399F1923019F002E0E5D8E0C7B0
:104F3000FE01FF9605A116A127A130A5003840E08B
:104F4000140740E0240740E03407E8F4E3EEFCE017
:104F500080819181FE01FF9605A116A127A130A5B0
:104F6000E3EEFCE00083118320DA002339F03ADB22
:104F7000A0E0BA2F1A2F0B2FE3D8BAC7E3EEFCE05C
:104F800080839183B5C701E0B7D8B2C72BE136E083
:104F90008E010E94F61D0023D1F1923019F002E03B
:104FA000ABD8A6C7FE01FF9605A116A127A130A583
:104FB000003840E0140740E0240740E0340720F5C3
:104FC000E3EEFCE080819181FE01FF9605A116A130
:104FD00027A130A5E3EEFCE000831183E6D900238E
:104FE00071F0E3EEFCE080839183FCDAA0E0BA2F5D
:104FF0001A2F0B2FA5D801E00093E50C79C7E3EE3B
:10500000FCE08083918374C701E076D871C728E5FE
:1050100036E08E010E94F61D0023E1F00091E50CC0
:10502000002389F000E068D80E94170F902F99356F
:1050300019F0993709F05CC704E110E00E94670C91
:1050400008E001BD55C704E110E00E94670C08E0CC
:1050500001BD4EC726E136E08E010E94F61D0023F9
:1050600019F10AE30E94E60D20E08E01085D1F4F52
:105070000E94C41F002361F000E00DAB9E01285D7B
:105080003F4F00EE19E00E94DE1D01E00093E50CA9
:10509000E2E1F6E11491E9E0F6E1049172D700EE65
:1050A00019E00E940A0F24C723E136E08E010E9416
:1050B000F61D002309F482C09130A9F580E08F31FC
:1050C00008F016C702E0809F00E0000E02E0101E0C
:1050D000F001E052F64F018105FF23C090E0FC0192
:1050E000EB58F64F00810023E1F021E018E1082F92
:1050F0000E94724D14E2082F18D722E0829F20E010
:10510000020E22E0121EF001E052F64F00831183DE
:10511000082F0E94473A182F00E01DDA182F00E0F0
:10512000F8D88395CCCF44245524E92FF0E031976B
:105130004E165F060CF0DCC6FE01EC59FF4F042D45
:1051400010E0000F111F000F111FE00FF11F008171
:10515000118122813381802F02E0809F00E0000EC8
:1051600002E0101EF001E052F64F018105FF24C05D
:10517000082F10E0F801EB58F64F00810023E1F012
:1051800021E018E1082F0E94724D14E2082FCDD6BD
:1051900022E0829F20E0020E22E0121EF001E05287
:1051A000F64F00831183082F0E94473A182F00E022
:1051B000D2D9182F00E0ADD84394B6CF2FE036E017
:1051C0008E010E94F61D002309F460C0913021F584
:1051D00080E08F3108F08CC690E0FC01EB58F64F70
:1051E00000810023B9F020E018E1082F0E94724DE1
:1051F00002E0809F00E0000E02E0101EF001E0528D
:10520000F64F018100620183182F00E0A4D9182F06
:1052100000E07FD88395DDCF44245524E92FF0E0CA
:1052200031974E165F060CF063C6FE01EC59FF4F36
:10523000042D10E0000F111F000F111FE00FF11FD0
:105240000081118122813381802F082F10E0F80125
:10525000EB58F64F00810023B9F020E018E1082F49
:105260000E94724D02E0809F00E0000E02E0101EDE
:10527000F001E052F64F018100620183182F00E037
:105280006AD9182F00E045D84394C7CF28E936E003
:105290008E010E94F61D002309F466C0913009F0CA
:1052A00048C00091090D1091080D011709F020C6A2
:1052B00008EC10E00E94670C0E94CE20E1E1F6E1CC
:1052C0001491E8E0F6E104915CD612E206E60E9451
:1052D0004D4D0E949E0E00E20E94E60D13E206E68E
:1052E0000E944D4D0E949E0E00E20E94E60D14E2C7
:1052F00006E60E944D4D0E949E0E0CE20E94E60DB5
:1053000012E205E60E944D4D0E949E0E00E20E94B0
:10531000E60D13E205E60E944D4D0E949E0E00E24E
:105320000E94E60D14E205E60E944D4D0E949E0E7D
:10533000B8CF923009F0DCC580E007C000E090E013
:10534000FC01E954F24F008383958F31B8F3FE01DD
:10535000FF9605A116A127A130A50093E20C0EE24D
:1053600015E10E940D4CC4C523E936E08E010E9470
:10537000F61D002339F421E936E08E010E94F61D66
:105380000023C1F0FE01FF9605A116A127A130A5BB
:10539000923021F002E00E947C20AAC5083020F063
:1053A00004E00E947C20A4C50093F40901E000936E
:1053B000E50C9EC52CE836E08E010E94F61D002308
:1053C00099F1933021F002E00E947C2091C5FE010A
:1053D000FF9605A116A127A130A5802FFE01FF96FB
:1053E00001A512A523A534A5902F983010F488307C
:1053F00020F004E00E947C207BC50AE30E94E60DB9
:10540000082F0E949E0E0DE20E94E60D0EE30E9400
:10541000E60D092F0E949E0E182F092F0E941B20B7
:1054200001E00093E50C64C528E735E08E010E9499
:10543000F61D002341F423E735E08E010E94F61D9E
:10544000002309F488C0933020F002E00E947C2001
:105450004FC5913019F40091F40906C0FE01FF9682
:1054600005A116A127A130A5073020F004E00E9475
:105470007C203EC5E3EEFCE020813181232B41F40A
:105480001091F409133020F004E00E947C2030C514
:10549000923039F417E00E941B2001E00093E50CE4
:1054A00019C09130A1F40091F409073080F417E09D
:1054B0000091F4090E941B20E0EEF9E004890395B5
:1054C000048B0E94E92001E00093E50C03C004E096
:1054D0000E947C20E3EEFCE000811181012B09F0A9
:1054E00007C50091F409013029F00091F409023058
:1054F00009F0FEC400E410E020E830E040EC50E0A9
:1055000080E01EC062E0869F020E131EF001E05292
:10551000F64F2080318062E0869F000E111EF00160
:10552000E052F64F60817181261A370A62E0869F49
:10553000040E151EF001E052F64F20823182839551
:105540008F3100F30E94CE2003E00E947C2002E015
:105550000E944E20CDC425E836E08E010E94F61D43
:10556000002339F428E036E08E010E94F61D002366
:10557000E9F1923029F5FE01FF9605A116A127A1B8
:1055800030A5802F873020F004E00E947C20B0C43A
:105590000091F409801770F4E0EEF9E004890A95AF
:1055A000048B0E94E92006C0182F1395082F0E9433
:1055B0001B2083958630C0F301E00093E50C98C46E
:1055C000913009F095C40091F409013058F0E0EEF3
:1055D000F9E004890A95048B0E94E92001E0009318
:1055E000E50C86C404E00E947C2082C42EE736E0ED
:1055F0008E010E94F61D002339F42CE736E08E015F
:105600000E94F61D002389F1FE01FF9605A116A157
:1056100027A130A5802F923021F002E00E947C204B
:1056200067C4873020F004E00E947C2061C406E05B
:10563000402E06C0142D1A95042D0E941B204A945A
:105640008415C0F317E0082F0E941B200091F40975
:10565000801738F4E0EEF9E004890395048B0E948A
:10566000E92001E00093E50C43C42AEB35E08E010C
:105670000E94F61D002379F0923048F0FE01FF965B
:1056800005A116A127A130A50E94604131C401E007
:105690000E9460412DC42AE435E08E010E94F61D6F
:1056A000002341F428E435E08E010E94F61D00231A
:1056B00009F461C0FE01FF9605A116A127A130A53E
:1056C000402E923021F002E00E947C2011C407E0BD
:1056D000401620F004E00E947C200AC499E580E096
:1056E0001DC0082F10E0F801EB58F64F0081002391
:1056F000A1F0042D10E040E450E00E94C34D22E0F0
:10570000829F000E111E00E4000E00E0101EF0014A
:10571000E052F64F018106FD9EE483958F3108F338
:105720000091F409401640F0993531F400E00E94F0
:105730007C200E94170F902F993519F0993709F0A6
:10574000D7C3E6E1F6E11491EDE0F6E1049119D456
:10575000042D0E949E0E07E00E944E20142D07E0AB
:105760000E941B2080E08F3108F0C2C3082F0E94E6
:10577000473A8395F8CF27E736E08E010E94F61D61
:10578000002309F4BAC0E3EEFCE040805180913080
:1057900061F4E3EEFCE00081118120E030E0FE01E5
:1057A000FF9605A316A327A330A7EFEDFDE0208108
:1057B0003181273302E0300738F023E333E012E28F
:1057C0000EEF0E947A4D06C02FEF33E012E20EEF8B
:1057D0000E947A4D00E010E0E3EEFCE000831183CC
:1057E00080E00CC022E0829F20E0020E22E0121E28
:1057F000F001E052F64F0083118383958F3100F55D
:1058000090E0FC01EB58F64F00810023B1F318E162
:10581000082F0E944D4D013021F41EE1082F85D341
:1058200003C014E2082F81D3003020E41207D1F620
:105830000DED1DE00E940D4C082F0E949E0EDDCF45
:10584000E3EEFCE040825182FE01FF9605A116A125
:1058500027A130A5A6D407C001E00093E60C05EF10
:105860001DE00E940D4C0091E80C0023A1F0009176
:10587000090D1091080D0117B1F30E94170F0B319C
:1058800059F30D3081F702E00093E60C0CEF1DE0B8
:105890000E940D4CE8CF0EE215E10E940D4C04EF82
:1058A00011E00E94670C80E00CC022E0829F20E0A3
:1058B000020E22E0121EF001E052F64F0083118327
:1058C00083958F31B0F490E0FC01EB58F64F0081E6
:1058D0000023B1F31EE1082F28D3003020E4120783
:1058E00021F70DED1DE00E940D4C082F0E949E0E29
:1058F000E7CF07E00E944E20FBC223E736E08E018F
:105900000E94F61D002309F457C0923051F4FE01A5
:10591000FF9605A116A127A130A5003024E01207AB
:1059200020F002E00E947C20E3C21A2F0B2F0E947D
:10593000AB221A2F0B2F0E941C210130E9F4FE012B
:10594000FF9605A116A127A130A5802F1A2F0B2F96
:105950000E943A21F801E052F64F80831A2F0B2F54
:105960000E943A21F801E052F64F00810E949E0EFB
:1059700001E00093E50CBCC2023009F0B9C2FE019F
:10598000FF9605A116A127A130A5C8011A2F0B2F3C
:105990000E943A21F801E052F64F808391831A2F3A
:1059A0000B2F0E948921BB2319F40A2F0E94473A2A
:1059B00001E00093E50C9CC22CE636E08E010E94CB
:1059C000F61D002341F42AE636E08E010E94F61D02
:1059D000002309F443C1BE01605F7F4FEDEDFDE997
:1059E00030E08B0148E150E00E94644E923071F447
:1059F000FE01FF9605A116A127A130A5073040E0C2
:105A0000140740E0240740E0340720F002E00E9441
:105A10007C206EC201E00093E50CFE01FF9605A11B
:105A200016A127A130A5102F07E00E941B2040E4FB
:105A300052EE60E070E080E03AC002E0809F8001BA
:105A4000212F220F220B322F040F151F261F371F65
:105A50000F5F1F4F2F4F3F4FF801322F3BBF069074
:105A600000E00BBF302C222402E0809F8001212F18
:105A7000220F220B322F040F151F261F371FF8018C
:105A8000322F3BBF0690202D00E00BBF30E0220DEF
:105A9000331D2F7F3370FE01E55CFE4F082F10E0B1
:105AA000000F111FE00FF11F2083318383958F3189
:105AB00020F2FE01FF9605A116A127A130A540E422
:105AC00050E00E94C34D005C1F4F80E026C022E0E2
:105AD000829F000E111E21E0020E20E0121EF00136
:105AE000E052F64F508140E022E0829F000E111EEE
:105AF000F001E052F64F208130E0240F351F2F7F58
:105B00003370FE01E350FF4F482F50E0440F551F04
:105B1000E40FF51F2083318383958F31C0F280E03D
:105B200068C0FE01E55CFE4F082F10E0000F111F5A
:105B3000E00FF11F208131812F7F33708E010350E0
:105B40001F4FFE01709690E0E80FF91F408150E072
:105B5000440F551F040F151FE02FF12F00811181F5
:105B60000F7F1370201B310B8E01055C1E4FFE0151
:105B7000709690E0E80FF91F408150E0440F551FE8
:105B8000040F151FE02FF12F008111810F7F13707B
:105B9000020F131F22E0829F20E0020E22E0121E5D
:105BA000F001E052F64F008311838E0103501F4F26
:105BB000FE01709690E0E80FF91F208130E0220F7F
:105BC000331F020F131FE02FF12F0081118100708E
:105BD0001C7F22E0829F20E0020E22E0121EF001D4
:105BE000E052F64F20813181202B312B20833183ED
:105BF00083958F3138F590E0FC01EB58F64F00812A
:105C00000023B1F3FE01709690E0E80FF91F0081C8
:105C10000F3F09F086CFFE01E350FF4F082F10E041
:105C2000000F111FE00FF11F0081118122E0829F00
:105C300020E0020E22E0121EF001E052F64F008337
:105C40001183D6CF07E00E944E2080E08F3108F00C
:105C50004FC1082F0E94473A8395F8CF26E636E0D9
:105C60008E010E94F61D0023C1F000E00E947C20FE
:105C70000E94170F093519F0093709F039C10E9440
:105C80006D220E94F222A0E0BA2F1A2F0B2F0E9441
:105C9000A02001E00093E50C2BC121E636E08E0147
:105CA0000E94F61D002341F42DE536E08E010E948E
:105CB000F61D002309F418C110E088242FEF3FE0FF
:105CC000A9010E94A54D22EF3FE0A9010E94B14D1C
:105CD00001E12FEF3FE0A9010E94B14D80E090E08B
:105CE00006C0FC01E052F64F0081100F0196803093
:105CF00002E09007B0F30091FF09011B0A950093A1
:105D0000FF090EE20E94E60D80E090E00BC0FC016E
:105D1000E052F64F00819C012050384FA9010E94AB
:105D2000B14D0196803002E0900788F300911E0C7F
:105D300020E03AE0A9010E94B14D00911F0C21E042
:105D40003AE0A9010E94B14D80E090E001C00196C7
:105D5000803002E0900770F49C012050384FA90178
:105D60000E94A54DFC01E052F64F1081011779F316
:105D700088248394E3EEFCE00081118125EF3FE06D
:105D8000A9010E94B14D882009F075C025EF3FE0C0
:105D9000A9010E94A54DE3EEFCE0208131810217AC
:105DA00009F069C00AEA24EF3FE0A9010E94B14D61
:105DB00008E001BD04EF11E00E94670C25EF3FE011
:105DC000A9010E94A54D10E0E3EEFCE000831183E1
:105DD000E3EEFCE0008111810F7F107000831183DE
:105DE00088240FEF24EF3FE0A9010E94B14DE3EEBC
:105DF000FCE00081118120E030E040E052E060E012
:105E000070E00E94044E2801390100E0400E00EECF
:105E1000501E00E0601E00E0701E80E090E001C0B7
:105E20000196803002E09007C0F49C012050384F6A
:105E3000A9010E94A54D602F8C0120E030E0040DE7
:105E4000151D261D371DF801322F3BBF069000E0BF
:105E50000BBF601529F302E0802E20E03AE0A90193
:105E60000E94A54D00931E0C21E03AE0A9010E947A
:105E7000A54D00931F0C8820F9F40E94D5210091B4
:105E8000F509002361F0E3EEFCE00081118120912F
:105E9000F50930E020503F4FA9010E94B14D0EE2BC
:105EA00015E10E940D4C0E94F222A0E0BA2F1A2F99
:105EB0000B2F0E94A02009C005ED1DE00E940D4C93
:105EC00000E3800E082D0E94E60D00E00093E50C33
:105ED00022EF3FE0A9010E94A54D2FEF3FE0A9016D
:105EE0000E94B14DAD9804C008EE1DE00E940D4C1B
:105EF0000091F409091599F00091F409013F20F08F
:105F000000E00093F40907C00091F409083018F08C
:105F100007E00093F4090E94E9209090F4091A2FF9
:105F20000B2F0E94AB220C94A1249A938A93802F6A
:105F3000082F0E945C4D0F3F2FEF120719F400E06D
:105F400012E01CC0E3EEFCE020813181232B51F0F4
:105F500090E0880F991FFC01E056F64F20813181B7
:105F6000021B130B212F27FF03C000E010E006C027
:105F7000003024E0120710F00FEF13E0899199919F
:105F800008959A938A93902F812F02E00E94E60D44
:105F90000BE10E94E60D0BE50E94E60D8A3038F019
:105FA000082F4AE00E94B54D005D0E94E60D082FC3
:105FB0004AE00E94B54D042F005D0E94E60D0BE300
:105FC0000E94E60D9A3038F0092F4AE00E94B54D44
:105FD000005D0E94E60D092F4AE00E94B54D042F96
:105FE000005D0E94E60D06E60E94E60D89919991FA
:105FF00008959A938A93FA93EA933A922A921A927C
:106000000A927A936A935A934A933A932A931A93E9
:106010000A938FB79BB700E00BBF78940091E80C10
:10602000002349F00091E70C002321F004E20E94D4
:10603000E60D01C0CED0EAEFFCE0008111810F5FD8
:106040001F4F008311830091260E102F139510937C
:10605000260E0F70002309F06EC0ECEFFCE000810B
:106060001181012B41F0ECEFFCE000811181015026
:106070001040008311830091F90C002349F0E9EFEF
:10608000FCE000810A95008308E015B3102715BBDA
:10609000AA9AA99A24B135B10091E70D10E00370D6
:1060A0001070000F111FF801E152F24F208331836D
:1060B000E7EEFDE0008103950083037007B90091CE
:1060C000270E102F13951093270E0770002399F5B4
:1060D000E6EDFDE00081039500830E94BC43879BB1
:1060E0002AC0969B28C00091F30C002321F5009153
:1060F0009A000F7700939A00959A96980FE113E013
:1061000001501040E9F700C0000000919B00102FE3
:1061100017FF0AC000919C00053531F404E110E03E
:106120000E94670C08E001BD969A959800919A002C
:10613000006800939A00E8EEFDE0008107FF0CC0C4
:106140000091260E002311F4A89815C00091260E88
:10615000083089F4A89A0FC00091260E1091E80D1E
:106160001023112341F40091E80D002321F001E0F8
:1061700015B3102715BB00E000931B0D9BBF8FBF0D
:10618000099119912991399149915991699179917F
:106190000990199029903990E991F99189919991F3
:1061A00018959A938A93C80120E030E010E20EEF30
:1061B0000E947A4DE5EFFCE08083918301E000933B
:1061C000F40C0093E80C00E00093E60C899199919F
:1061D00008950E94774E24970091F40C002309F44F
:1061E0004DC000E00093691000E010E0EFE5F0E141
:1061F00000831183EDE5F0E100831183E1E6F0E136
:106200000083118300E00093B00C03E0009367105B
:10621000CC2431C002E0C09E800100501E4FF80126
:10622000E052F64F208131810C2D10E0000F111F3C
:10623000F801EC5CF04F2083318300E010E02C2D5E
:1062400030E0220F331FF901E650F04F0083118335
:106250002C2D30E0220F331FF901E45DF14F008354
:1062600011832C2D30E0220F331FF901E854F04F39
:1062700000831183C3940FE1C01660F2EDE5F0E1F5
:1062800000811181EFE5F0E12081318102171307D0
:1062900008F00CC3EDE5F0E1008111810F5F1F4FA5
:1062A00000831183E2EEFCE0008100FF86C0EAEF8C
:1062B000FCE0008111810370002309F059C002E263
:1062C0000093A00703E00093A10722E012E006E696
:1062D0000E94E94A002331F0009127081091280814
:1062E0009091290800916A10000F00936A10EAE665
:1062F000F0E1008101FF08C09B3068F0EAE6F0E1C0
:1063000000810160008307C0933328F0EAE6F0E1E2
:1063100000810160008302E20093A00703E0009384
:10632000A10722E012E005E60E94E94A002331F0CD
:1063300000912708109128088091290800916B107E
:10634000000F00936B10EBE6F0E1008101FF08C045
:106350008B3098F1EBE6F0E10081016000832DC005
:10636000833358F1EBE6F0E100810160008325C042
:10637000EAEFFCE0008111810370013061F408E272
:106380000093A00704E00093A10722E012E007E6D3
:106390000E94E94A12C0EAEFFCE00081118103701B
:1063A000023059F404E30093A00704E00093A1072E
:1063B00022E012E007E60E94E94A009167100330EC
:1063C00009F474C280E00CE190E0FC01E056F84F63
:1063D0000083839504E090E0FC01E056F84F0083D1
:1063E0008395CC244CC001E010E02C2D30E0205EE1
:1063F0003F4FF901EF55F34F408142954F700E9496
:10640000D34D90E0FC01E056F84F0083839501E006
:1064100010E02C2D30E0205E3F4FF901EF55F34F97
:1064200040814F700E94D34D90E0FC01E056F84F40
:106430000083839502E0C09E00E0000E02E0101E83
:10644000F001E052F64F0081118190E0FC01E0562E
:10645000F84F0083839502E0C09E00E0000E02E04A
:10646000101EF001E052F64F00811181012F10E063
:1064700090E0FC01E056F84F00838395C3940FE150
:10648000C01608F00EC2DD24F601EB58F64F00816D
:106490000023A1F300916710002309F092C00C2D96
:1064A00010E0000F111FF801EA58F04F0081118130
:1064B0002C2D30E0220F331FF901E854F04F2081DA
:1064C0003181021B130B212F220F220B322FEDE5FE
:1064D000F0E14081518160E070E00E94044EEFE500
:1064E000F0E14081518160E070E00E944E4E2C2D21
:1064F00030E0220F331FF901E854F04F4081518101
:10650000400F511F2C2D30E0220F331FF901E650B0
:10651000F04F408351832C2D30E0220F331FF901BF
:10652000E854F04F2081318115950795020F131F14
:10653000212F220F220B322FEDE5F0E14081518116
:1065400060E070E00E94044E40E950E060E070E0DE
:106550000E94044E4FE050E060E070E00E944E4E1A
:10656000012F122F232F330F330B259517950795E6
:106570002C2D30E0220F331FF901E055F14F00833D
:1065800011830C2D10E0000F111FF801EE50F14F98
:10659000208131810C2D10E0000F111FF801E05512
:1065A000F14F00811181020F131F22E0C29E20E0F3
:1065B000020E22E0121EF001E052F64F008311831A
:1065C00010C100916710013009F046C00C2D10E099
:1065D000000F111FF801EE50F14FA081B1810C2D79
:1065E00010E0000F111FF801E259F14F00811181F5
:1065F000212F220F220B322FEDE5F0E14081518156
:1066000060E070E00E94044EEFE5F0E140815181CE
:1066100060E070E00E944E4E0A0F1B1F22E0C29EF7
:1066200020E0020E22E0121EF001E052F64F00833D
:1066300011830C2D10E0000F111FF801EA58F04FE4
:10664000208131810C2D10E0000F111FF801E65060
:10665000F04F20833183C5C0DD24F601E45CFF4E9A
:106660000081002309F078C00C2D10E0000F111FED
:10667000F801E854F04F0081118111950195104007
:10668000212F220F220B322FEDE5F0E140815181C5
:1066900060E070E00E94044EEFE5F0E1408151813E
:1066A00060E070E00E944E4E2C2D30E0220F331F30
:1066B000F901E854F04F40815181400F511F2C2DBA
:1066C00030E0220F331FF901E650F04F4083518331
:1066D0002C2D30E0220F331FF901EE50F14FA08135
:1066E000B1812C2D30E0220F331FF901E854F04F17
:1066F0002081318115950795020F131F212F220F3D
:10670000220B322FEDE5F0E14081518160E070E035
:106710000E94044E40E950E060E070E00E94044EA8
:106720004FE050E060E070E00E944E4E012F122FCB
:10673000232F330F330B2595179507950A0F1B1F32
:1067400022E0C29E20E0020E22E0121EF001E05282
:10675000F64F0083118345C00C2D10E0000F111F70
:10676000F801EE50F14FA081B1810C2D10E0000F27
:10677000111FF801E259F14F00811181212F220FE1
:10678000220B322FEDE5F0E14081518160E070E0B5
:106790000E94044EEFE5F0E14081518160E070E03D
:1067A0000E944E4E0A0F1B1F22E0C29E20E0020EE6
:1067B00022E0121EF001E052F64F008311830C2DEF
:1067C00010E0000F111FF801EA58F04F20813181CD
:1067D0000C2D10E0000F111FF801E650F04F208340
:1067E000318302E0C09E00E0000E02E0101EF001C6
:1067F000E052F64F018107FF0EC000E010E022E0FA
:10680000C29E20E0020E22E0121EF001E052F64F7E
:10681000008311831CC002E0C09E00E0000E02E075
:10682000101EF001E052F64F20813181203004E04B
:10683000300768F00FEF13E022E0C29E20E0020E66
:1068400022E0121EF001E052F64F0083118390E027
:10685000FC01E056F84FC0828395E2EEFCE0008137
:1068600000FFC1CD00916A100F3F19F004E1C0167E
:1068700049F000916B100F3F09F4B5CD05E1C0164A
:1068800009F0B1CD00E890E0FC01E056F84F00833C
:10689000839500E890E0FC01E056F84F0083839573
:1068A000C9CD282F13E80EEF0E946E4A009169109F
:1068B000002321F000E00093E80CE5C5EDE5F0E1F0
:1068C00000811181EFE5F0E120813181021713078A
:1068D00008F4D9C500E010E0EDE5F0E10083118394
:1068E000CC2427C002E0C09E00E0000E02E0101E93
:1068F000F001E052F64F208131810C2D10E0000FA5
:10690000111FF801EE50F14F208331830C2D10E060
:10691000000F111FF801E650F04F208131810C2D3E
:1069200010E0000F111FF801E854F04F208331836D
:10693000C3940FE1C016B0F200916710002309F074
:106940009FC001E000936710E3E6F0E10081118150
:10695000E5E6F0E120813181220F331F021B130B8A
:10696000EFE5F0E100831183CC2446C00C2D10E04C
:10697000000F111FF801E45DF14F808191810C2D12
:1069800010E0000F111FF801E055F14F0081118157
:10699000801B910B0C2D10E0000F111FF801EA581D
:1069A000F04F00811181212F220F220B322FE5E6BB
:1069B000F0E14081518160E070E00E94044E4CE0C3
:1069C00050E060E070E00E94044E45E050E060E07E
:1069D00070E00E944E4E012F122F232F330F330BE6
:1069E000801B910B0C2D10E0000F111FF801E259D4
:1069F000F14F80839183C3940FE1C01608F0D6C095
:106A0000DD24F601E45CFF4E0081013009F0AECFD9
:106A10000C2D10E0000F111FF801E45DF14F008113
:106A200011812C2D30E0220F331FF901E055F14F79
:106A300020813181021B130B212F220F220B322FB9
:106A4000EFE5F0E14081518160E070E00E94044E8A
:106A5000E3E6F0E140815181E5E6F0E1608171819A
:106A6000461B570B60E070E00E944E4E2C2D30E02C
:106A7000220F331FF901E259F14F00831183BBCF7D
:106A8000009167100130D1F502E000936710E5E650
:106A9000F0E100811181EFE5F0E100831183CC2466
:106AA0000FE1C01608F082C00C2D10E0000F111F7E
:106AB000F801E45DF14F208131810C2D10E0000FD1
:106AC000111FF801E259F14F00811181201B310B98
:106AD0000C2D10E0000F111FF801E055F14F00815F
:106AE0001181201B310B0C2D10E0000F111FF8013C
:106AF000E259F14F20833183C394D2CF00916710C4
:106B00000230B1F4E1E6F0E100811181012B61F086
:106B100003E000936710E1E6F0E100811181EFE509
:106B2000F0E10083118342C000E0009367103EC093
:106B3000009167100330D1F5CC2432C002E0C09E32
:106B400000E0000E02E0101EF001E052F64F20813E
:106B500031810C2D10E0000F111FF801EC5CF04F9B
:106B60002083318300E010E02C2D30E0220F331F12
:106B7000F901E650F04F008311832C2D30E0220FF5
:106B8000331FF901E45DF14F008311832C2D30E0B8
:106B9000220F331FF901E854F04F00831183C3948F
:106BA0000FE1C01658F200E00093671000916710E3
:106BB000002309F068C4E8E6F0E100810395008352
:106BC000009168101091B50C011728F40091F40C95
:106BD000002309F4DFC00091F40C002399F5E5EFE0
:106BE000FCE000811181E7EFFCE00083118300915C
:106BF000B00C002329F0E1EAFCE007850A9507873D
:106C00000091B00C0023F1F40091E60C013039F44E
:106C100000E010E0E5EFFCE00083118313C0009179
:106C2000E60C023041F40091BB0C10E0E5EFFCE013
:106C30000083118307C00091BA0C10E0E5EFFCE07F
:106C400000831183E5EFFCE000811181012B21F429
:106C500001E0009369109EC000E00093F40CE3EEA5
:106C6000FCE000811181E5EFFCE020813181021719
:106C7000130741F500E010E020E030E0E8E2FEE03C
:106C800000831183228333830091B00C002309F029
:106C900053C0ADE0B0E0A03400E0B00708F04CC055
:106CA000E8E2FEE000811181228133810A0F1B1F7F
:106CB000F801E052F64F0081FD01EF55F34F0083DC
:106CC0001196E9CFE5EFFCE00081118120E030E092
:106CD000322F212F102F00E0110F221F331F0050E1
:106CE00010422F4F3F4FE8E2FEE0008311832283E2
:106CF00033830091B00C0023F9F4ADE0B0E018C08C
:106D0000E8E2FEE040815181628173818D0120E0E3
:106D100030E0040F151F261F371FF801322F3BBF2D
:106D2000069000E00BBFFD01EF55F34F0082119676
:106D3000A03400E0B00720F3E8E2FEE0008111811A
:106D400022813381005C1F4F2F4F3F4F00831183FF
:106D5000228333830091B50C083020F40091B50CE8
:106D6000002381F40BE01DE00E940D4CE5EFFCE0F8
:106D7000008111810E94ED0E0DE50E94E60D01E0FB
:106D8000009369100091B00C002309F428CF00E0B3
:106D900000936810A0E0B0E020C0E8E2FEE00081CF
:106DA000118122813381A801B9014F5F5F4F6F4F7D
:106DB0007F4FE8E2FEE04083518362837383F801F2
:106DC000322F3BBF069000E00BBF8D01005C1D4FD2
:106DD000F801E052F64F00821196A03400E0B007AF
:106DE00058F5E3EEFCE000811181E5EFFCE0208145
:106DF00031810217130789F6E8E2FEE00081118174
:106E000022813381F801E052F64F20818D01005C30
:106E10001D4FF801E052F64F2083E8E2FEE00081CA
:106E20001181228133810F5F1F4F2F4F3F4F00830E
:106E3000118322833383D0CF009168100395E5EF4F
:106E4000FCE0808191811091B50C011708F459C0C4
:106E50000091E60C013039F400E010E0E5EFFCE0D1
:106E60000083118315C00091E60C023031F400E07C
:106E70000093B00C8091BB0C0BC00091B00C0230A1
:106E800028F0E5EFFCE08081918102C08091BA0C8E
:106E900090E0E3EEFCE0008111818017910759F446
:106EA00000E410E020E030E0E8E2FEE0008311833F
:106EB0002283338326C0882379F4E8E2FEE0008150
:106EC00011812281338100541040204030400083E2
:106ED00011832283338315C0082F10E020E030E0B7
:106EE000322F212F102F00E0110F221F331F005CC3
:106EF0001F412F4F3F4FE8E2FEE0008311832283C2
:106F00003383A0E0B0E01BC0E8E2FEE040815181A5
:106F1000628173818D0120E030E0040F151F261F70
:106F2000371FF801322F3BBF069000E00BBF8D01E9
:106F300000581D4FF801E052F64F00821196A03420
:106F400000E0B007D0F4E3EEFCE00081118180178F
:106F5000D9F6E8E2FEE000811181228133810A0F37
:106F60001B1FF801E052F64F20818D0100581D4F84
:106F7000F801E052F64F2083E1CF00916910002321
:106F800009F081C200915E0C10E045E00E94D34DF3
:106F90004091B70C50E00E94DF4DE1E6F0E1008344
:106FA000118300915F0C1091B70C019F800145E0A7
:106FB0000E94D94DD8010A2F0B2B11F4A1E0B0E0AB
:106FC00020E030E0CC240EC00C2D10E0000F111F8B
:106FD000F801E45DF14F008111812017310708F4B9
:106FE0009801C3940FE1C01608F0FCC0DD24F6013F
:106FF000EB58F64F00810023A1F30C2D10E0000F99
:10700000111FF801EC5CF04F4081518102E0C09EFD
:1070100000E0000E02E0101EF001E052F64F408347
:1070200051830C2D10E0000F111FF801EE50F14FAD
:107030004083518300E010E04C2D50E0440F551F79
:10704000FA01E055F14F0083118302E0C09E00E495
:10705000000E02E0101EF001E052F64F0081118197
:107060004C2D50E0440F551FFA01E056F64F608159
:107070007181DD24F601E954F24F4081542F550F00
:10708000550B460F571F040F151F412F47FF03C015
:1070900000E010E006C0003044E0140710F00FEFED
:1070A00013E04C2D50E0440F551FFA01EC5CF04FFB
:1070B00040815181B801641B750B4C2D50E0440F89
:1070C000551FFA01E45DF14F608371834C2D50E050
:1070D000440F551FFA01EC5CF04F608171814C2D1B
:1070E00050E0440F551FFA01EC5CF04F0083118310
:1070F00042E0C49E40E8040E42E0141EF001E0525B
:10710000F64F208031804C2D50E0440F551FFA017E
:10711000E056F64F00801180020C131CDD24F601AE
:10712000E954F24F4081542F550F550B400D511D1E
:10713000052E07FE03C040E050E006C04030E4E00A
:107140005E0710F04FEF53E06017710718F4041753
:10715000150730F00617170728F44017510710F4E9
:1071600000E001C001E0002391F4E1E6F0E10081DC
:107170001181012B61F40091681010E0E091B50CD1
:10718000F0E031970E171F074CF0882339F400E028
:10719000DD24F601E45CFF4E008306C001E0DD243F
:1071A000F601E45CFF4E00830091B10C0A3009F453
:1071B00018CF0C2D10E0000F111FF801E45DF14F06
:1071C0004081518155230AF0FFCE0C2D10E0000FB5
:1071D000111FF801E45DF14F0081118111950195B6
:1071E0001040FBCE0091B10C0A3029F4E3E6F0E147
:1071F000A083B18313C0890148E250E00E94C34DCF
:10720000C8018D0143E050E00E94C34DA8018C01EC
:107210000E94DF4DE3E6F0E1008311830091B90C99
:1072200010E0E5E6F0E100831183E5E6F0E100819E
:107230001181000F111FE3E6F0E120813181021777
:107240001307E8F1E2E7F9E0008102FF13C00BE564
:107250000E94E60D009168100E94CF0D0CE20E9482
:10726000E60DE3E6F0E1008111810E94ED0E0DE5EF
:107270000E94E60DE3E6F0E100811181012B39F473
:1072800000E010E0E5E6F0E10083118318C0E3E6DA
:10729000F0E1008111810150104016950795E5E657
:1072A000F0E100831183E5E6F0E100811181012B1B
:1072B00031F400E010E0E3E6F0E100831183E3E65F
:1072C000F0E10081118120E030E0000F111F221F4A
:1072D000331FE5E6F0E180819181A0E0B0E0880F06
:1072E000991FAA1FBB1F081B190B2A0B3B0B480138
:1072F0005901880C991CAA1CBB1C880E991EAA1E39
:10730000BB1E000F111F221F331F088319832A83FE
:107310003B83082D09290A290B2929F49924AA2439
:10732000BB2488248394088119812A813B81012B05
:10733000022B032B41F401E010E020E030E0088351
:1073400019832A833B83CC2442C0041915092609DA
:107350003709A401B5010E944E4E2C2D30E0220FBA
:10736000331FF901EA58F04F008311830C2D10E010
:10737000000F111FF801EA58F04F208131812030B1
:1073800004E030075CF00FEF13E02C2D30E0220F0B
:10739000331FF901EA58F04F008311830C2D10E0E0
:1073A000000F111FF801EA58F04F20813181213080
:1073B0000CEF30075CF401E01CEF2C2D30E0220FC5
:1073C000331FF901EA58F04F00831183C3940FE192
:1073D000C01608F050C00C2D10E0000F111FF8016E
:1073E000E854F04F00811181212F220F220B322F00
:1073F000AC01BD010E94044E280139010C2D10E0A2
:10740000000F111FF801E45DF14F00811181212F60
:10741000220F220B322F0801190140E05AE060E0F0
:1074200070E0800191010E94044E080119014CE0B6
:1074300050E060E070E0800191010E944E4EDD243A
:10744000F601E45CFF4E4081442309F07ECF04192D
:10745000150926093709488159816A817B810E9473
:107460004E4E2C2D30E0220F331FF901EA58F04F19
:10747000008311837BCFE5E6F0E100811181EFE528
:10748000F0E1008311832496EEE00C94884E0E9474
:107490007F4E402E5524F201EB58F64F0081002319
:1074A00009F47EC002E0409E800100501E4FF801AA
:1074B000E052F64F018105FF06C020E018E1042DDF
:1074C0000E94724D6DC0E3EEFCE000811181012B42
:1074D000C9F002E0409E00E0000E02E0101EF00144
:1074E000E052F64F008111810F7F1370242D30E0A0
:1074F000220F331FF901E056F64FA081B181A00F92
:10750000B11F0DC002E0409E00E0000E02E0101E20
:10751000F001E052F64FA081B181AF7FB3700B2F25
:1075200007FF03C0A0E0B0E006C0A03004E0B00751
:1075300010F0AFEFB3E014E2042D0E945C4D0F3F5A
:1075400023E0120758F4A017B10720F40A1B1B0B05
:10755000C80106C0CD01801B910B02C008E010E0FD
:107560009695879596958795883000E0900710F45A
:1075700088E090E00EE10093A0070A2F0093A10796
:10758000AB2FB0E0A093A207082F0093A307892F89
:1075900090E08093A40725E013E0042D0E94E94ABF
:1075A000E6E00C94904E0E94814ED8010091E80CC8
:1075B000002309F041C00A2F0B2BF1F1A03800E0A5
:1075C000B007D0F500E010E0E3EEFCE000831183AB
:1075D00080E00BC022E0829F900120503E4FF901D5
:1075E000E052F64F0083118383958F3110F590E0C0
:1075F000FC01EB58F64F00810023B1F318E1082F8E
:107600000E944D4D013029F41EE1082F0E94952F54
:1076100004C014E2082F0E94952F003020E41207C6
:10762000C9F60DED1DE00E940D4C082F0E94CF0DF4
:10763000DBCF8D010E94D130E4E00C94924E6AC001
:107640000E94170F1091FF0C163018F010E01093E5
:10765000FF0C2091FF0C30E0F901E050F34F008364
:10766000EFEFFCE0108113951083053551F5009183
:10767000FF0C0250073008F00A5F10E0F801E050FC
:10768000F34F00810F3FE9F400E00093FF0C0FEF90
:107690002091FF0C30E0F901E050F34F0083EFEF51
:1076A000FCE000810395008305E52091FF0C30E0AC
:1076B000F901E050F34F0083EFEFFCE00081039508
:1076C00000830091FF0C063029F50091000D0F3F5B
:1076D00009F50091010D0535E9F40091020D1091B5
:1076E000030D10950117B1F40091040D1091050DD3
:1076F0001095011779F401E00093FE0C3091040D10
:1077000020E00091020D10E0020F131FE9EEFCE0F3
:10771000008311830091090D1091080D011709F0E4
:107720008FCF08959A938A93C901083C09F0CFC07E
:10773000183151F4082F092B21F402E00093E60CD4
:1077400001C18C0130DFFEC01A3111F01B3149F547
:10775000EBEEFCE0808391830FEF0E94E60D05E5E0
:107760000E94E60DEBEEFCE0008111810E94E60D27
:10777000EBEEFCE00081118100950E94E60DEBEE3E
:10778000FCE000811181012F10E00E94E60DEBEE7C
:10779000FCE000811181012F10E000950E94E60DB0
:1077A000D1C01F3159F4882311F401E001C000E079
:1077B000102F10FDAB9A10FFAB98C4C01232A1F588
:1077C00040E050E010E020E030E000E00E94BC0C1F
:1077D000002309F4B7C0EFEEFCE000811181081727
:1077E000190739F040E050E010E09C0101E00E94F0
:1077F000BC0CE2E6F9E0038114810817190709F4CB
:10780000A1C0E2E6F9E083839483082F23E030E00F
:10781000A9010E94B14D892F90E0082F24E030E0AB
:10782000A9010E94B14D8EC0113229F4ECEFFCE0A9
:107830008083918387C0153221F48C010E94670EEA
:1078400081C0163251F48C010E94670E0DE00E9437
:10785000E60D0AE00E94E60D75C01832A1F540E081
:1078600050E010E020E030E000E00E94BC0C00237B
:1078700009F468C0E1EFFCE00081118108171907E5
:1078800039F0AC0110E020E030E004E00E94BC0CD4
:10789000E2E6F9E0018512850817190709F452C0DC
:1078A000E2E6F9E081879287082F29E030E0A9011C
:1078B0000E94B14D892F90E0082F2AE030E0A90105
:1078C0000E94B14D3FC002E010E8D5D43BC0043661
:1078D000F0F00D36E0F42091E80C222339F021E09D
:1078E00020931B0D20911B0D2223E1F7E2E5F7E128
:1078F000212F30E0E20FF31F2491223021F49C016C
:107900000E947A4D1FC0282F0E94724D1BC02091EB
:10791000E80C222339F021E020931B0D20911B0D50
:107920002223E1F7EAE1F7E1212F30E0E20FF31F34
:107930002491223021F49C010E947A4D03C0282F0B
:107940000E94724D899199910895083C09F0E4C014
:10795000183181F4E5EFFCE000811181012B29F45D
:10796000E7EFFCE0008111810895E5EFFCE0008184
:1079700011810895193121F40091E80C10E0089567
:107980001A3111F01B3129F4EBEEFCE0008111817A
:1079900008951C3111F01D3149F451DE00E00093CF
:1079A000FE0CE9EEFCE00081118108951E3129F4FE
:1079B00046DE0091FE0C10E008951F3141F405B33E
:1079C0000695069506950095017010E0089512320F
:1079D000B1F540E050E010E020E030E000E00E942F
:1079E000BC0C002339F1E2E6F9E003811481EFEEEB
:1079F000FCE02081318102171307E1F0EFEEFCE09B
:107A000000811181E2E6F9E003831483EFEEFCE0EC
:107A10000081118123E030E0A9010E94B14DEFEE19
:107A2000FCE000811181012F10E024E030E0A90189
:107A30000E94B14DE2E6F9E0038114810895143209
:107A400069F440E050E010E020E030E000E00E9407
:107A5000BC0CEDEEFCE00081118108951032B9F408
:107A600000E0809902C0006111E00C9902C008603A
:107A700011E00D9902C0046011E00E9902C002608D
:107A800011E00F9902C0016011E010E00895113279
:107A900029F4ECEFFCE00081118108951832B1F572
:107AA00040E050E010E020E030E000E00E94BC0C3C
:107AB000002339F1E2E6F9E001851285E1EFFCE00F
:107AC0002081318102171307E1F0E1EFFCE0008132
:107AD0001181E2E6F9E001871287E1EFFCE0008125
:107AE000118129E030E0A9010E94B14DE1EFFCE0F5
:107AF00000811181012F10E02AE030E0A9010E94ED
:107B0000B14DE2E6F9E001851285089501E010E843
:107B1000B2D30FEF1FEF08950436E8F00E36D8F415
:107B20002091E80C222339F021E020931B0D2091B5
:107B30001B0D2223E1F7E2E5F7E1212F30E0E20F10
:107B4000F31F2491223019F40E945C4D08950E9485
:107B50004D4D10E008950F31D8F42091E80C222308
:107B600039F021E020931B0D20911B0D2223E1F71A
:107B7000EAE1F7E1212F30E0E20FF31F24912230F8
:107B800019F40E945C4D08950E944D4D10E0089537
:107B900000E010E008959A938A93ECE1FDE0008103
:107BA000118198012F5F3F4FECE1FDE0208331838D
:107BB00020E030E0005010462F4F3F4FF801322FA9
:107BC0003BBF0690002D10E01BBFECE1FDE04081C3
:107BD00051819A012F5F3F4FECE1FDE0208331831B
:107BE00060E070E0405050466F4F7F4FFA01362FF3
:107BF0003BBF0690202D10E01BBFECE1FDE0408173
:107C00005181CA010196ECE1FDE08083918360E03F
:107C100070E0405050466F4F7F4FFA01362F3BBF08
:107C2000069010E01BBF002321F4102D022F8DDEE3
:107C30004EC0023061F4102D30E0220F331FF901E5
:107C4000E85DF24F20813181022F7FDE40C001309C
:107C500069F4002D10E0000F111FF801E85DF24FEC
:107C600000811181102F022F70DE31C00330A9F482
:107C7000002D10E0000F111FF801E85DF24F0081A8
:107C80001181102F30E0220F331FF901E85DF24F10
:107C900020813181022F59DE1AC0043039F4502D71
:107CA00040E0022F10E0040F151F11C0053069F4E9
:107CB000102D00E030E0200F311F220F331FF9019B
:107CC000E85DF24F0081118102C000E010E089916F
:107CD000999108950E94814EA801ECE1FDE0008198
:107CE000118198012F5F3F4FECE1FDE0208331834C
:107CF00020E030E0005010462F4F3F4FF801322F68
:107D00003BBF0690002D10E01BBFECE1FDE00080C2
:107D10001180C0010196ECE1FDE080839183C001F8
:107D2000A0E0B0E080509046AF4FBF4FFC013A2F2B
:107D30003BBF0690602D10E01BBFECE1FDE0008032
:107D40001180C0010196ECE1FDE080839183C001C8
:107D5000A0E0B0E080509046AF4FBF4FFC013A2FFB
:107D60003BBF069010E01BBF002329F49A01102DA1
:107D7000062FD8DC4BC0023069F49A01102D70E058
:107D8000660F771FFB01E85DF24F40815181042FA0
:107D9000C9DC3CC0013071F49A01002D10E0000FE5
:107DA000111FF801E85DF24F00811181102F062F9D
:107DB000B9DC2CC00330B1F49A01002D10E0000FA3
:107DC000111FF801E85DF24F00811181102F70E062
:107DD000660F771FFB01E85DF24F40815181042F50
:107DE000A1DC14C0043021F407E010E044D20EC03E
:107DF000053061F4102D00E070E0600F711F660F18
:107E0000771FFB01E85DF24F40835183E4E00C945F
:107E1000924EC1DEEEE1FDE000831183ECE1FDE076
:107E20000081118198012F5F3F4FECE1FDE020833D
:107E3000318320E030E0005010462F4F3F4FF801D3
:107E4000322F3BBF069000E00BBF0092240DA3DE53
:107E5000E0E2FDE0008311830091240D002379F41A
:107E6000EEE1FDE000811181E0E2FDE02081318161
:107E70000217130711F401E0089500E0089500913E
:107E8000240D013079F4E0E2FDE000811181EEE1A2
:107E9000FDE0208131810217130710F401E00895FD
:107EA00000E008950091240D023079F4EEE1FDE048
:107EB00000811181E0E2FDE020813181021713078A
:107EC00010F001E0089500E008950091240D0330C2
:107ED00079F4EEE1FDE000811181E0E2FDE0208136
:107EE00031810217130710F401E0089500E00895AE
:107EF0000091240D043079F4E0E2FDE0008111816D
:107F0000EEE1FDE0208131810217130710F001E05E
:107F1000089500E008950091240D053079F4EEE114
:107F2000FDE000811181E0E2FDE020813181021756
:107F3000130711F001E0089500E0089505E010E056
:107F40009AD100E008950091250D013061F400916F
:107F5000270D002331F00091260D002311F001E0E0
:107F6000089500E008950091250D023061F400911C
:107F7000270D002321F40091260D002311F001E0CC
:107F8000089500E0089506E010E075D100E008953E
:107F90009A938A930230C9F0ECE1FDE0408151816F
:107FA0009A012F5F3F4FECE1FDE02083318360E0D9
:107FB00070E0405050466F4F7F4FFA01362F3BBF65
:107FC000069010E01BBF0092230D1091230D1F5F40
:107FD00009F440C1125091F01A9509F11A9509F46B
:107FE0004CC01A9509F4F2C01A9509F4FBC01A9511
:107FF00009F407C11A9509F41CC137C1002331F0F7
:10800000CADDECE1FDE00083118332C1ECE1FDE06B
:10801000008111810D5F1F4F0083118329C100234F
:1080200019F1ECE1FDE0008111810D5F1F4F00832C
:108030001183B1DDE0E2FDE000831183ECE1FDE0BE
:10804000008111810650104000831183E0E2FDE0C1
:10805000008111813FDEECE1FDE0008111810D5FC7
:108060001F4F0083118304C1ECE1FDE00081118109
:108070000A5F1F4F00831183FBC0002309F49DC0DA
:10808000ECE1FDE0008111810D5F1F4F0083118342
:1080900082DDEEE1FDE000831183ECE1FDE0008193
:1080A000118198012F5F3F4FECE1FDE02083318388
:1080B00020E030E0005010462F4F3F4FF801322FA4
:1080C0003BBF069000E00BBF0092240D64DDE0E2B0
:1080D000FDE0008311830091240D002359F4EEE1AB
:1080E000FDE000811181E0E2FDE080819181800F5F
:1080F000911F50C00091240D013059F4EEE1FDE0D4
:1081000080819181E0E2FDE000811181801B910B73
:1081100041C00091240D023061F4EEE1FDE00081E8
:108120001181E0E2FDE0408151810E94C34DC80110
:1081300031C00091240D033061F4EEE1FDE00081D7
:108140001181E0E2FDE0408151810E94DF4DC801D4
:1081500021C00091240D003159F4EEE1FDE00081D1
:108160001181E0E2FDE0808191818023912312C0A2
:108170000091240D013159F4EEE1FDE000811181FF
:10818000E0E2FDE080819181802B912B03C004E02F
:1081900010E071D0ECE1FDE0008111810A50104047
:1081A000008311838C0196DDECE1FDE000811181FB
:1081B000095F1F4F008311835BC0ECE1FDE000818C
:1081C0001181065F1F4F0083118352C0002309F005
:1081D0004FC0ECE1FDE000811181ECE1FDE00083A6
:1081E000118346C0002321F00BE10093220D40C013
:1081F000ECE1FDE000811181ECE1FDE00083118301
:1082000037C0002369F0ECE1FDE0008111810D5FD2
:108210001F4F61D2C0DCECE1FDE00083118328C078
:10822000ECE1FDE0008111810D5F1F4F00831183A0
:108230001FC0002331F079D2ECE1FDE0008311830F
:1082400017C0ECE1FDE000811181ECE1FDE000836D
:1082500011830EC0002361F4ECE1FDE00081118187
:10826000ECE1FDE00083118303C003E110E003D0E3
:108270008991999108959A938A93C801E2E7F9E068
:10828000008101FF1AC001E715E10E940D4C8C012D
:108290000E94ED0E0BE50E94E60DECE1FDE0008191
:1082A00011810E94ED0E0AE30E94E60D0091230D5C
:1082B0000E94CF0D0DE50E94E60D899199910895D8
:1082C0000E94824EA02FAA2311F49598969A00E05E
:1082D00010E0ECE1FDE00083118380E090E204E037
:1082E0000093230DAA2321F002E315E10E940D4C17
:1082F00000E00093220D05C002E04ADEAA2309F047
:1083000013D10091220D0B3109F407C1ECE1FDE01E
:1083100020813181203000EC300708F0FEC0009150
:10832000230D053009F4F9C0ECE1FDE00081118175
:108330000817190708F0F1C0ECE1FDE00081118198
:1083400098012F5F3F4FECE1FDE02083318320E077
:1083500030E0005010462F4F3F4FF801322F3BBF07
:10836000069000E00BBF0092230DE3E2FDE00081E8
:1083700007FFC2CF0091230D005849F00A9509F478
:108380006FC00A9509F4B0C00A95B1F1C2C041DDD1
:108390000093260D0091260D0093270DECE1FDE0E2
:1083A0000081118198012F5F3F4FECE1FDE02083B8
:1083B000318320E030E0005010462F4F3F4FF8014E
:1083C000322F3BBF069000E00BBF0092250DAA2381
:1083D00009F0AAD00091250D002309F092CF009159
:1083E000270DD6DDAA2309F48CCF0091270D002399
:1083F00009F487CF99D085CF0CDD0093260DA3DD3E
:108400000093270DECE1FDE00081118198012F5FC1
:108410003F4FECE1FDE02083318320E030E000506D
:1084200010462F4F3F4FF801322F3BBF069000E020
:108430000BBF0092250DAA2309F076D00091250DDF
:10844000002309F05ECF0091270DA2DDAA2309F4D5
:1084500058CF0091270D002309F453CF65D051CF99
:108460000091270D002359F0ECE1FDE0008111811E
:10847000085F1F4F0083118300E08ADD42CFC9DC13
:108480000093260D0091260D0093270DECE1FDE0F1
:108490000081118198012F5F3F4FECE1FDE02083C7
:1084A000318320E030E0005010462F4F3F4FF8015D
:1084B000322F3BBF069000E00BBF0092250DAA2390
:1084C00009F032D00091250D002309F01ACF009158
:1084D000270D5EDDAA2309F414CF0091270D002398
:1084E00009F40FCF21D00DCFAA2309F01DD00091A0
:1084F000270D002311F401E001C000E049DDAA23AB
:1085000009F4FFCE0091270D002309F0FACE0CD01C
:10851000F8CE00E110E0AFDEF4CE0091E80C0023CD
:10852000E1F7E3E00C94934E0CE810E00E940D4C50
:1085300066D00DE20E94E60D0091230D0E94CF0D42
:108540000AE30E94E60D00E20E94E60D0091260D6E
:108550000E94CF0D0DE30E94E60D08E20E94E60D99
:10856000EEE1FDE0008111810E94ED0E0CE20E941F
:10857000E60D00E20E94E60D0091240D0E94CF0D51
:108580000CE20E94E60D00E20E94E60DE0E2FDE052
:10859000008111810E94ED0E09E20E94E60D00E2C9
:1085A0000E94E60D0091250D0E94CF0D0BE70E9461
:1085B000E60D0091270D0E94CF0D0DE70E94E60DFC
:1085C0000BE50E94E60DECE1FDE0008111810E94C7
:1085D000ED0E0DE50E94E60D0E94170F0093220D8F
:1085E0000091220D0B3151F404E615E10E940D4C6F
:1085F000ECE1FDE0008111810E94ED0E08950091F3
:10860000230D003829F40BE715E10E940D4C089565
:108610000091230D013829F403E815E10E940D4C67
:1086200008950091230D023829F40BE815E10E940A
:108630000D4C08950091230D033829F403E915E149
:108640000E940D4C08950091230D013029F40BE98F
:1086500015E10E940D4C08950091230D023029F47C
:1086600003EA15E10E940D4C08950091230D03309B
:1086700029F40BEA15E10E940D4C08950091230D99
:10868000043029F403EB15E10E940D4C089500918C
:10869000230D053029F40BEB15E10E940D4C0895D4
:1086A0000091230D063029F403EC15E10E940D4CD6
:1086B00008950091230D073029F40BEC15E10E9479
:1086C0000D4C08950091230D0F3F21F403ED15E1AA
:1086D0000E940D4C08952091B60D2A3010F520917E
:1086E000B60D30E0220F331FF901E457F24F00833B
:1086F0001183E6EBFDE00081039500832091270DB7
:1087000030E00091B60D10E0000F111FF801E457A2
:10871000F24F20833183E6EBFDE000810395008377
:10872000089509E010E0A7DD08950091B60D00233B
:10873000E9F0E6EBFDE000810A95008310E0000F10
:10874000111FF801E457F24F008111810093270DAA
:10875000E6EBFDE000810A95008310E0000F111F99
:10876000F801E457F24F0081118108950AE010E00A
:1087700082DD0FEF1FEF08950E94814E00916C1073
:10878000002309F0D3C000916909013009F094C0B9
:10879000EFEDFDE002811381012B09F45AC000E0E6
:1087A0000093D60D00E010E0EBEDFDE000831183B7
:1087B00000E010E0EDE6F0E10083118301E00093BA
:1087C0006C10EFEDFDE00081118145E050E00E946A
:1087D000DF4D10E0E7EDFDE000831183E7EDFDE004
:1087E00080819181EFEDFDE00281138145E050E051
:1087F0000E94DF4D10E0801B910BE9EDFDE08083CE
:108800009183E9EDFDE020813181243700E03007DC
:1088100020F003E00093E80D27C2E9EDFDE02081A0
:108820003181223700E0300720F007E00093E80DA7
:108830001BC2E9EDFDE020813181203700E03007E7
:1088400020F00FE00093E80D0FC20FE00093E80D59
:108850000BC20091D60D0370002309F005C2EFEDA5
:10886000FDE00081118145E050E00E94DF4D10E005
:10887000E7EDFDE000831183E7EDFDE0808191816C
:10888000EFEDFDE00281138145E050E00E94DF4DF5
:1088900010E0801B910BE9EDFDE080839183E9ED11
:1088A000FDE020813181293500E0300708F0DCC18E
:1088B0000FE70093E80DD8C1EFEDFDE002811381D1
:1088C000012B09F0D1C10091D60D0370002309F0EE
:1088D000CBC1EFEDFDE00081118145E050E00E9449
:1088E000DF4D10E0E7EDFDE000831183E7EDFDE0F3
:1088F00080819181EFEDFDE00281138145E050E040
:108900000E94DF4D10E0801B910BE9EDFDE08083BC
:108910009183E9EDFDE020813181293500E03007C8
:1089200008F0A2C10FE70093E80D9EC100916C1002
:10893000013009F04AC1EFEDFDE002811381012B06
:1089400061F400E010E01BBD0ABD00E00093E80DFB
:10895000A89800E000936C1087C10091D60D0F71AC
:10896000002329F400E010E01BBD0ABD7DC1009189
:10897000D60D0F71023009F077C1EFEDFDE00081F7
:10898000118145E050E00E94DF4D10E0E7EDFDE091
:1089900000831183E7EDFDE080819181EFEDFDE043
:1089A0000281138145E050E00E94DF4D10E0801B02
:1089B000910BE9EDFDE080839183EBEDFDE000811B
:1089C0001181E9EDFDE0208131810217130740F4A8
:1089D000E9EDFDE000811181EBEDFDE00083118305
:1089E000EAE1F6E1A3EEBDE00D911C911197169519
:1089F000079516950795E00FF11F049110E0EDED36
:108A0000FDE000831183E9EDFDE0008111810A5F43
:108A10001F4FE7EDFDE0208131810217130718F0A9
:108A20000FEF13E010C00AEF17E1E7EDFDE0408122
:108A30005181E9EDFDE020813181421B530B46500D
:108A400050400E94DF4D003024E0120710F00FEF7D
:108A500013E01BBD0ABDADEDBDE0ED91FC9111979A
:108A6000F69720F003E00093E80D32C0ADEDBDE0D5
:108A7000ED91FC911197F49720F007E00093E80D39
:108A800027C0E9EDFDE020813181243700E0300787
:108A900020F003E00093E80D1BC0E9EDFDE020812C
:108AA0003181223700E0300720F007E00093E80D25
:108AB0000FC0E9EDFDE020813181203700E0300773
:108AC00020F00FE00093E80D03C00FE00093E80DE5
:108AD000EDE6F0E1008111810F5F1F4F00831183EC
:108AE000EDE6F0E120813181283601E0300758F0D1
:108AF00000E010E01BBD0ABD0FEF0093E80D02E897
:108B000000936C10B1C0E9EDFDE020813181263782
:108B100000E0300758F000E010E01BBD0ABD0FEF89
:108B20000093E80D01E800936C109EC0EBEDFDE0B2
:108B3000008111810C531040E9EDFDE0208131816D
:108B40000217130798F0E9EDFDE020813181253609
:108B500000E0300758F000E010E01BBD0ABD0FEF49
:108B60000093E80D03E800936C107EC0EDEDFDE08E
:108B7000208131812C3300E0300758F000E010E014
:108B80001BBD0ABD0FEF0093E80D04E800936C10C5
:108B90006BC0ADEDBDE0ED91FC911197F89708F435
:108BA00063C0E9EDFDE020813181203700E030072E
:108BB00008F45AC000E010E01BBD0ABD0FEF00939F
:108BC000E80D04E800936C104FC000916909023071
:108BD00041F002E00093690927E030E0A9010E941A
:108BE000B14DEFEDFDE002811381012BC1F400E0F6
:108BF00010E01BBD0ABD00E00093E80DA89800E05E
:108C000000936C1000916909002371F100E000935A
:108C1000690927E030E0A9010E94B14D25C000910B
:108C2000D60D0F71002301F5EFEDFDE000811181FC
:108C300045E050E00E94DF4D10E0E7EDFDE00083ED
:108C40001183E7EDFDE080819181EFEDFDE0028190
:108C5000138145E050E00E94DF4D10E0801B910B36
:108C6000E9EDFDE080839183E4E00C94924E07EE01
:108C700006B900E010E01BBD0ABD03EC0FBD02E029
:108C80000EBD03E00093E70DE7EEFDE000810395E4
:108C90000083037007B901E010E00E94670C24B163
:108CA00035B10091E70D10E003701070000F111F37
:108CB000F801E152F24F20833183E7EEFDE00081BD
:108CC00003950083037007B901E010E00E94670C70
:108CD00024B135B10091E70D10E003701070000F62
:108CE000111FF801E152F24F20833183E7EEFDE0DE
:108CF000008103950083037007B901E010E00E9432
:108D0000670C24B135B10091E70D10E003701070CD
:108D1000000F111FF801E152F24F20833183E7EE7B
:108D2000FDE0008103950083037007B901E010E0C6
:108D30000E94670C24B135B10091E70D10E003707B
:108D40001070000F111FF801E152F24F20833183A0
:108D500008950E94824E1A981B9A0E94E30BA898CD
:108D600000E0009370090093710900E0009372091C
:108D70000093730900E00093E80C00E00093F90C05
:108D800022E030E0A9010E94A54D0F3FA9F021E0AB
:108D900030E0A9010E94A54D0F3F71F023EF3FE0A5
:108DA000A9010E94A54D033038F427E030E0A90165
:108DB0000E94A54D033048F101E00093630921E0D2
:108DC00030E0A9010E94B14D02E20093620920E067
:108DD00030E0A9010E94B14D00E022E030E0A9019D
:108DE0000E94B14D80E023EF3FE0082FA9010E94CF
:108DF000B14D0AE00093F90C00E00093690927E007
:108E000030E0A9010E94B14D37C021E030E0A90156
:108E10000E94A54D0093630920E030E0A9010E9463
:108E2000A54D0093620923EF3FE0A9010E94A54DE3
:108E3000802F23E030E0A9010E94A54D0093650931
:108E400024E030E0A9010E94A54D0093660929E0C5
:108E500030E0A9010E94A54D00936B092AE030E0A3
:108E6000A9010E94A54D00936C0927E030E0A901FB
:108E70000E94A54D0093690900E000936A0911E082
:108E800020E830E000E00E94C40B21E0109162096C
:108E900000E00E94330C21E012E201E00E94330C5A
:108EA00000E00093700900937109E1DE789424EFEB
:108EB0003FE0A9010E94A54D053519F400E0C8D492
:108EC0005EC1833038F080E023EF3FE0082FA90136
:108ED0000E94B14D94B700E004BF21EF3FE0A9012B
:108EE0000E94A54D002361F0923051F483958330A8
:108EF00008F080E023EF3FE0082FA9010E94B14D68
:108F00009A70992361F400916909002341F000E00F
:108F10000093690927E030E0A9010E94B14D21EFDB
:108F20003FE0A9010E94A54D013031F001E021EFA1
:108F30003FE0A9010E94B14D00916909023009F09A
:108F40005DC000E800936C100FEF0093E80D56C071
:108F500090E0809B04C002E310E00E94670C009147
:108F6000090D1091080D011769F00E94170FA02F2D
:108F7000A53521F40091080D0093090D082F0E94DA
:108F8000E60D01C0A0E0882311F4AC9807C0813041
:108F900011F4AD9803C0823009F4AE98933209F011
:108FA00046C0A33209F043C004E110E00E94670C00
:108FB00008E001BD809B04C002E310E00E94670C42
:108FC0000C991CC002E310E00E94670C0091690933
:108FD000002371F4EFEDFDE002811381012B41F0DC
:108FE00001E00093690927E030E0A9010E94B14D3A
:108FF0000C9BFECF02E310E00E94670C809B31C007
:10900000AD9AAC9AAE9A0091090D1091080D011716
:1090100009F49ECF0E94170F902F953521F40091EF
:10902000080D0093090D082F0E94E60D92CF99308C
:1090300011F0A93089F404E110E00E94670C08E007
:1090400001BD8395833008F080E023EF3FE0082FD7
:10905000A9010E94B14DAECF9D3019F0AD3009F09D
:10906000A9CF21EF3FE0A9010E94A54D002331F0D7
:1090700000E021EF3FE0A9010E94B14D809BFECFAF
:1090800004E110E00E94670C00E910E0C6D38ED323
:10909000882391F401E0DCD3902F0CE810E0BDD3DD
:1090A000092F0E942B0F08E512E0B7D301E00093CF
:1090B00072090E943B0FFDCF00916209013059F106
:1090C00001E0009362092091620914E00EEF0AD5D5
:1090D00005E912E0A2D300E814E82EE130E0409167
:1090E000620950E060E070E04F5F5F4F6F4F7F4F6D
:1090F0000E944E4E0E940E0E00EB12E08ED30091A5
:10910000620920E030E0A9010E94B14D09B904EFE5
:1091100011E00E94670C01E010E0E3EEFCE0008348
:10912000118301E095D3902F0CE810E076D3092F3E
:109130000E942B0F08E512E070D307E0009372093C
:109140000E94D521EFEDFDE020813181273302E03F
:10915000300730F023E333E012E20EEFCBD405C04A
:109160002FEF33E012E20EEFC5D4813071F401E04D
:1091700010E0E3EEFCE0008311830E94F22203E0A2
:10918000009372090E94732416C08230A1F404E691
:1091900010E00E94670C02E00093720900E00E9458
:1091A000604104E610E00E94670C04E110E00E94B8
:1091B000670C08E001BDFFCFFA93EA934A933A9314
:1091C0002A931A930A933FB74BB700E00BBFAA98B4
:1091D00020919C000091080D10E00F701070F801B4
:1091E000E65FF24F2083E8E0FDE000810395008315
:1091F0004BBF3FBF09911991299139914991E9914B
:10920000F9911895FA93EA934A933A932A931A9309
:109210000A933FB74BB700E00BBF00917009102FC6
:109220001395109370092CB110E0F801E056F94F36
:1092300020834BBF3FBF09911991299139914991E1
:10924000E991F99118952497AA98A99808EA10E04D
:10925000E4D223C00E94170F0E94E20D5E9A009193
:10926000090D1091080D0117A9F75E9BFECF1A9802
:109270001B9A0091710910917009011771F000910A
:10928000710910E0F801E056F94F0081E1E7F9E0DB
:109290001081139510830E94E60D0091090D109125
:1092A000080D011731F31B981A9AD9CF0E947E4EF0
:1092B000AA98A99808EA10E0B0D218C05E9BFECF29
:1092C0001A981B9A0091710910917009011771F099
:1092D0000091710910E0F801E056F94F0081E1E7D3
:1092E000F9E01081139510830E94E60D0091090D9D
:1092F0001091080D011731F31B981A9A1CC0FC013C
:109300003A2F3BBF0690002D10E01BBF8F5F9F4F91
:10931000AF4FBF4F600E0E94E20D5E9A01E0400E1B
:1093200000E0501E0FEF401607E1500640F3062DF7
:109330000E94E20D5E9A0091090D1091080D01172F
:1093400009F4BCCF0E94170F0E3741F480E090EC77
:10935000A0E0B0E0662444245524E4CF0E94E20D4E
:109360005E9AE9CF0E94804E902F44249F3F29F4BB
:1093700000E014EF21E030E004C008EE13E020E04C
:1093800030E080E013C04091710950E0FA01E056EE
:10939000F94F4081E1E7F9E0508153955083682F00
:1093A00070E0FB01EE5DF74F408383958917D8F499
:1093B00040E050E060E070E00090710910907009AA
:1093C000011479F40A011B01A001B1014F5F5F4F45
:1093D0006F4F7F4F001511052205330568F74424B0
:1093E0004394442081F2A82FB0E00091D8080E3FAA
:1093F00009F470C0442071F09F3F61F0E2E7F9E0AA
:10940000008100FF03C00FE11DE007D20091700949
:1094100000937109A43008F45DC0009122080F3F49
:1094200021F4009123080F3F71F0E2E7F9E0008199
:1094300000FF03C004E31DE0F0D100917009009328
:10944000710900E048C0009124081091D808011764
:1094500071F0E2E7F9E0008100FF03C00AE41DE0DB
:10946000DCD1009170090093710900E034C02091B3
:10947000250830E00A2F10E0045010402017310773
:1094800071F0E2E7F9E0008100FF03C000E61DE0B3
:10949000C4D1009170090093710900E01CC082E002
:1094A00007C090E0FC01EE5DF74F0081B00F83959F
:1094B0008A17B8F3BF3F71F0E2E7F9E0008100FFDF
:1094C00003C006E71DE0A9D100917009009371095E
:1094D00000E001C00A2FE5E00C94914E0E94814EFD
:1094E0003FEF3093D6083FEF3093D7080093D8086A
:1094F000022F0E5F0093D9081093DA0880E00DC0A8
:1095000090E0FC01E056F84F0081A82FB0E01596DE
:10951000FD01EA52F74F00838395821788F300E03C
:109520002A5FA22F82E007C090E0FC01EA52F74FC9
:109530001081010F839590E0EA2FF0E031978E17AC
:109540009F0794F3009590E0FC01EA52F74F0083E7
:109550001B981A9A80E009C05E9A90E0FC01EA52DA
:10956000F74F00810E94E20D83958A17A8F35E9B56
:10957000FECF1A981B9A0A2FE4E00C94924E0E9498
:10958000814ED801922F992359F40091D8080E3FAB
:1095900021F400EF11E041D103C001E112E03DD11F
:1095A00080E00CC0082F10E0FD01E00FF11F0081EA
:1095B0000E949E0E00E20E94E60D8395891790F3AB
:1095C00001E412E02AD1092F0E942B0FE4E00C9451
:1095D000924E0E947F4E802F912F422E01E00093E9
:1095E000E70CB0E02DC040E050E060E070E0F0E05B
:1095F0008A019B01A801B9014F5F5F4F6F4F7F4FF9
:10960000083EE3E01E07E0E02E07E0E03E0798F4A6
:109610000091710910917009011751F300917009BF
:109620000093710940E050E060E070E00F2FF02FF0
:10963000F3950536E8F20091700900937109B3952E
:10964000B23008F051C00091700900937109242DC7
:10965000192F082F43DFA02F913061F48E3F29F49A
:1096600055245A945092740930C006E0502E5092FE
:1096700074092BC0923039F45090A10706E0500EC7
:109680005092740922C08E3FC1F08F3140F4082FF0
:1096900010E0F801EB58F64F0081023870F0843684
:1096A00080F08E3670F4082F10E004561040F80158
:1096B000EB56F64F0081023820F45524509274097D
:1096C00013C006E0502E50927409552009F4B7CF0C
:1096D000052D48DE0093740900917409051521F0E9
:1096E0000FEF501609F07FCF00E00093E70C0091D8
:1096F0007409051509F443C00091D8080E3FF9F12B
:10970000E2E7F9E0008100FF15C00DED1DE085D016
:10971000082F0E942B0F07EB10E07FD02A2F06EDB9
:1097200018E02DDF09EC10E078D02091740902E2F6
:1097300018E025DFE2E7F9E0008101FF1EC000E04C
:1097400011E80E943B41082F0E949E0E00E20E94F9
:10975000E60D092F0E949E0E00E20E94E60D009188
:10976000A0070E949E0E00E20E94E60D0091A10754
:109770000E949E0E00E20E94E60D00E014C00091DF
:109780007309002379F007EB10E047D02A2F06ED8C
:1097900018E0F5DE09EC10E040D02091740902E2F7
:1097A00018E0EDDE01E0E6E00C94904E0BED10E0E9
:1097B00034D000E814E82EE130E04091990050E008
:1097C00060E070E04F5F5F4F6F4F7F4F0E944E4EE3
:1097D0000E940E0E00E20E94E60D00EB12E01DD08A
:1097E0000CE20E94E60D05EE10E017D000E814E848
:1097F0002EE130E049B150E060E070E04F5F5F4F34
:109800006F4F7F4F0E944E4E0E940E0E00E20E944C
:10981000E60D00EB12E001D00895EF97EF97A497C3
:1098200020E001C02395203A60F430E0F801E20F17
:10983000F31F4491FE0130E0E20FF31F4083442305
:1098400089F78E010E940A0FEF96EF96A49608956D
:109850000E94814EA02FAA2361F00CE810E0DDDF0A
:1098600009E40E94E60D04E40E94E60D0AE30E946A
:10987000E60D90E080E00EC0843658F08E3648F455
:1098800020E0082F10E004561040F801EB56F64F88
:1098900020838395803888F520E011E0082F99DE39
:1098A000002309F18F3140F420E8082F10E0F8017F
:1098B000EB58F64F20830DC0843658F08E3648F4AE
:1098C00020E8082F10E004561040F801EB56F64F40
:1098D0002083AA2331F0082F0E949E0E00E20E94EE
:1098E000E60D9395D6CF8F3138F620E0082F10E0A3
:1098F000F801EB58F64F2083CCCF40EC50EE60E0FF
:1099000070E080E059C002E0809F8001212F220F8B
:10991000220B322F040F151F261F371F0F5F1F4FFB
:109920002F4F3F4FF801322F3BBF0690102D00E024
:109930000BBF00E022E0829F212C220C2208322C57
:10994000040E151E261E371EF001322D3BBF069059
:1099500020E02BBF1124000E111E082F10E0000F75
:10996000111FF801E056F64F00821182082F10E017
:10997000000F111FF801E056F64F20813181203091
:1099800000E4300769F0082F10E0000F111FF80104
:10999000E056F64F20813181203000E4300759F441
:1099A00000E010E0282F30E0220F331FF901E056CD
:1099B000F64F0083118383958F3108F4A4CF80E0A4
:1099C00012C014E2082F0E94952F0060106222E05E
:1099D000829F20E0020E22E0121EF001E052F64FBC
:1099E0000083118383958F3180F5082F10E0F801F3
:1099F000EB58F64F00810023A9F310E1082F4DD05A
:109A00000068282F30E0F901EB58F64F008315E08D
:109A1000082F43D0002321F020E015E0082F62D06A
:109A200018E1082F3AD0013061F61EE1082F0E949C
:109A3000952F22E0829F20E0020E22E0121EF0010C
:109A4000E052F64F00831183CDCF84E620C0A82FCB
:109A5000B0E0A456B040FD01EB56F64F0081002364
:109A6000A9F010E1082F19D00068A82FB0E0A45683
:109A7000B040FD01EB56F64F008315E0082F0DD0E6
:109A8000002321F020E015E0082F2CD083958E369E
:109A9000F0F2092FE4E00C94924E1093A00711E02D
:109AA0001093A10722E012E094DD002319F0009149
:109AB000270808950FEF08951093A00712E0109360
:109AC000A10722E012E085DD002349F0309128084B
:109AD00020E00091270810E0020F131F08950FEFF8
:109AE0001FEF08951093A0072093A10722E013E031
:109AF00070DD08951093A007122F1093A107232F54
:109B000030E02093A20723E013E063DD08950FE324
:109B10000DBF05E00EBFC0E0D5E00E949D4E0023C2
:109B200011F00E94AF4E00E00BBF0E94A9460E94B8
:109B3000D24E0C94D24EE199FECF08954F5F5F4F05
:109B4000FADF4EBB5FBBE09A0895FADF0DB30895CC
:109B50004F5F5F4F4EBB5FBBF894E29AE19A0FBE36
:109B600008950FB6E8DF0DBBF5CF0024E8E0EA95D5
:109B700032F0001F001C0416D0F3041AF8CF001FA7
:109B8000402D00950895002411240030010741F074
:109B90001695079510F4040E151E440F551FF5CFAA
:109BA000002D112D08954A951AF0000F111FFBCFBB
:109BB00008954A951AF016950795FBCF089500244D
:109BC0001124EFE0001F111F001C111C04161506C4
:109BD00010F0041A150AEA95AAF7001F111F402D6C
:109BE000512D00951095089530952095109501956B
:109BF0001F4F2F4F3F4F0895709560955095419599
:109C00005F4F6F4F7F4F0895002411242224332487
:109C1000E02FE12BE22BE32B71F03695279517957A
:109C2000079520F4040E151E261E371E440F551FDF
:109C3000661F771FEDCF002D112D222D332D089596
:109C40004A952AF0000F111F221F331FF9CF0895E4
:109C50000024112422243324E0E2EA9592F0001F2C
:109C6000111F221F331F001C111C221C331C041641
:109C700015062606370688F3041A150A260A370A37
:109C8000ECCF001F111F221F331F402D512D622DBD
:109C9000732D00951095209530950895FF27772313
:109CA0001AF4F1600E94FC4D33231AF4F0950E94DF
:109CB000F44D0E94284EF69510F40E94F44DF6954E
:109CC00010F40C94FC4D0895AF93BF93B12FA02FC7
:109CD0003BBFD895EF5FFF4F3F4F0D924150504033
:109CE000B9F74BBFBF91AF910895FA92EA92DA9219
:109CF000CA92BA92AA929A928A927A926A925A9244
:109D00004A92BA93AA939A938A930895FF84EE8411
:109D1000DD84CC84BB84AA84998488847F806E800F
:109D20005D804C80BB81AA8199818881F0E00FB66B
:109D3000F894CE0FDF1F0FBE089501E0089520E0D4
:109D400002D0E9F708952D9301501040202F212BC8
:109D500008953BBF27913BB7F6DFD9F7089505EF8C
:109D60001DE92801F20130E03BBF07911691F20195
:109D70003296A791B691F201349647915791669128
:109D8000242F252B262B21F0FA01362FE2DF01C0EC
:109D9000D6DF07E0400E00E0501EA20143305E49CE
:109DA00008F3089500008895FECF141A1F24292E69
:109DB00033383D4D151B20252A2F34390808080952
:109DC0000909090909090909090909090909090903
:109DD0000808080808080808080808070700FF031B
:109DE000020504070609080B0A0D0C0F0E111013CB
:109DF000121514FF0060014005039E00CF09A00664
:109E000000000049440050494E47004700474F00BA
:109E100044524553455400524553455400535953F9
:109E20005F57520041435400414354494F4E005242
:109E300045475F5752005700575200575249544503
:109E40000053594E435F5752005357520043414C01
:109E50005500444543004845580043414C430043A6
:109E6000414C440052000D0A205B4349443A005DD6
:109E700020005245540052455455524E0052554E02
:109E80000048454C50004C004C544F535300540074
:109E9000544F5353004349440054455354004348DE
:109EA0004B0044454D4F004D4F4E49544F520042D8
:109EB00041554400534541524348004C45440053EA
:109EC00043414E0055504441544500440044554DD3
:109ED00050004F4646004F4E004E414D4500434F07
:109EE0005059005000504147450042004245464FFE
:109EF0005245004E004E45585400474F544F004DB8
:109F00004F4E0052450053504545440054494D457D
:109F1000005244005245414400480045584954000D
:109F20005341560053415645004E4557004D004D94
:109F30004952524F520053455400504C4159004928
:109F400000494E534552540044454C455445004D3C
:109F50004F5645005300535445500042414C414E2A
:039F600043450076
:00000001FF
